:020000040000FA
:040000006CEF14F09D
:08000800ABEF14F0166E7F0B44
:1000100016BC8008F76A240FF66E0800F55016BE6D
:1000200000081200000306090C101316191C1F22E9
:1000300025282B2E313336393C3F414447494C4E1D
:10004000515355585A5C5E60626466686A6B6D6FA6
:1000500070717374757678797A7A7B7C7D7D7E7E1B
:100060007E7F7F7F7F002A6A2B6A01D01E6E1F5021
:100070001E5ED8A01F062B502A5ED8A02B06D89053
:100080001F321E32D8902B322A32031C1A6E041CE7
:100090001B6E1A2AD8B41B2A830E256E266A276A7D
:1000A000286A296A246A0F0EEA6E02C0E9FF071C5B
:1000B0007DEC02F000D000D004001E502626D8B0FF
:1000C000272A1F5027262A502826D8B0292A2B5005
:1000D000292627509BDF800F176E295097DF800F4E
:1000E00017261730242602C0E9FFEF500710D8A0CA
:1000F0000718EF6E2504D8B4830E256ED8B41A2ADB
:10010000D8B41B3ED7D71200066A800E326E89EF34
:1001100000F01E6A1F6A206A216A089A9AEC01F0B0
:10012000D30FD8B4088A2D0FC60FF8E20A0FF6E3F2
:100130001A6E196A186A176A0A0E166E5BEC02F0DC
:100140001A5016241E6E17501F6E000ED8B0010EE6
:100150001F261850206E000ED8B0010E2026195010
:10016000216E000ED8B0010E2126060606E09AEC9C
:1001700001F0C60F02E20A0FDBE208AA0BD01E1E36
:100180001F1E201E211E1E2AD8B41F2AD8B4202AC2
:10019000D8B4212A1E501200066A1E6E1F6A0096ED
:1001A0000650D8B40086050E056E270E1B6E100E85
:1001B0000CD8030E1B6EE80E08D81B6A640E05D817
:1001C0001B6A0A0E02D81E5008D01A6E1F50176EF6
:1001D0001E50166E44EC02F01650166E054E009638
:1001E000065003E0055CD8B008D01650D8A400969D
:1001F00000B603D0300F90EF01F01200346E2BAE3A
:1002000003D02D0E90EC01F00E6A0F6A106A116A8D
:100210002B8E6A0E2A26D8902B322C322D32113298
:1002200010320F320E322A3EF6D72D502A5C2D2680
:100230002A5E2C502B5C2C262B5E066A3AD82E0E9A
:1002400090EC01F0356AD8900E342D6E0F342C6E80
:1002500010342B6E11342A6E3536D8902D362C364C
:100260002B362A3635360E502D260F50D8B00F3C7F
:100270002C261050D8B0103C2B261150D8B0113C71
:100280002A26D8B0353ED8902D362C362B362A3635
:1002900035363550300F90EC01F02DC00EF02CC0EB
:1002A0000FF02BC010F02AC011F0342ECBD7D8900D
:1002B00012000096065003E100860A0E066E2DC05D
:1002C00019F02CC018F02BC017F02AC016F0056AE0
:1002D000216A206A1F6A0A0E1E6EE7EC01F0052AE9
:1002E0000550065CD8A4F4D71E50D8A4009600A6EA
:1002F00002D0062C04D01E50300F90EC01F0062ED8
:10030000DED71200A66AA68E0900F55002E002D8D8
:10031000FBD7120004009EA8FDD7AD6ED880120056
:1003200001B48AEF01F001A205D001B003D001B2FF
:10033000EE6E120032BEEE501200AA6AA96EA66AD4
:10034000A680A850A94AAA2A1200AA6AA86EA66A7C
:10035000A684550EA76EAA0EA76EA6820400A6B2AA
:10036000FDD7A694A94AAA2A1200E836E8363C0B23
:100370000109C212C009C216C050F80B0209C06EB2
:10038000320ED9EC01F0C2820400C2B2FDD7C4CF54
:100390002BF0C3502A6E12001B6A1A6EFF0E1A262B
:1003A0001B2200D0D8A01200030E176EE70E02D851
:1003B000F5D7176AFD0F166EFF0E00D001D0162676
:1003C000040000D0D8A01726D8A01200F8D71950E2
:1003D0002118800BF46E19AE06D0D880000E165688
:1003E00017561856195621AE06D0D880000E1E5644
:1003F0001F56205621561A6A1B6A1C6A1D6A2E6AED
:100400002F6A306A316A215020101F101E1023E01D
:10041000200EF36ED89016361736183619362E364B
:100420002F36303631361E502E5C1F502F5820503C
:1004300030582150315809E31E502E5E1F502F5A5C
:100440002050305A2150315AD8801A361B361C366B
:100450001D36F32EDFD7F4AE06D0D880000E1A5624
:100460001B561C561D561AC016F01BC017F01CC098
:1004700018F01DC019F02EC01EF02FC01FF030C0A4
:1004800020F031C021F012001F6A1E6A100EF36EB8
:1004900017341E361F361A501E5C1B501F5805E3BA
:1004A0001A501E5E1B501F5AD88016361736F32E70
:1004B000EFD716501200200E226E2E6A2F6A306A75
:1004C000316AD89016A00ED01E502E261F50D8B0DC
:1004D0001F3C2F262050D8B0203C30262150D8B0C9
:1004E000213C3126313230322F322E32193218323D
:1004F00017321632222EE5D71200E988E92AEC16C7
:100500001200A66AA68E0900F55002E0EE6EFBD737
:100510001200F34E02D0E652FCD7E6CFEEFFE82EF3
:10052000FCD71200E466FED7F36EE552F32EFDD73A
:10053000E6CFEEFFE82EFCD71200610EE75C05E681
:100540007B0EE75C02E7DF0EE716E650EE6EF5E1A4
:100550001200A66AA68EEE500900F55C02E1F5666F
:10056000FAD7120013500F18386E38BE30D013BEB1
:1005700017D012500E5CD8A0000CD8A4010C135058
:100580000F5CD8A0000CD8A4010C1450105CD8A0AB
:10059000000CD8A4010C1550115CD8A0000C010C63
:1005A0000E50125CD8A0000CD8A4010C0F50135CA4
:1005B000D8A0000CD8A4010C1050145CD8A0000CDA
:1005C000D8A4010C1150155CD8A0000C010C0FAE82
:1005D000010C000C13500F18386E38BE34D013BE07
:1005E00019D012500E5CD8A0000CD8A4010C1350E6
:1005F0000F5CD8A0000CD8A4010C1450105CD8A03B
:10060000000CD8A4010C1550115CD8A0000CD8A483
:10061000010C000C0E50125CD8A0000CD8A4010CE8
:100620000F50135CD8A0000CD8A4010C1050145C1F
:10063000D8A0000CD8A4010C1150155CD8A0000C57
:10064000D8A4010C000C0FAE010C000C12500E5C73
:10065000356E19E2356C0EC037F012C00EF037C09F
:1006600012F00FC037F013C00FF037C013F010C0F6
:1006700037F014C010F037C014F011C037F015C0B7
:1006800011F037C015F01A0E356078D0125276E0AE
:10069000346A0F50376E1318396E0F8E138E080E92
:1006A000355E08E315C034F014C015F013C014F023
:1006B000136AF5D7352607E0D89013321432153275
:1006C0003432352EF9D739AE35D01550115E14506D
:1006D000105A13500F5A07E2D880000E11561056C8
:1006E0000F56800E371A346C04E01106000E105AB3
:1006F0000F5A040E356E0F660DD010C00FF011C0EA
:1007000010F034C011F0346A080E0E5E2DE3352E61
:10071000F2D72AD00FBE08D0D89034361136103612
:100720000F360E2EF7D720D036AC26D034AE24D0DC
:10073000346A11D0155011261450102213500F2274
:1007400006E30F321032113234320E4A0FD036AC7B
:1007500013D034AE11D0113E0FD0103E0DD00F3E4D
:100760000BD0D8801190EDD70E6A02D036820E6879
:10077000116A106A800E0F6E37AE0F9E1150120074
:100780000F50306E1318396E125053E00E5254E071
:100790000E5E7F0E03E20E2603E24DD00E264EE2E1
:1007A00011C02EF010C02FF0308E138E180E376E41
:1007B000116A106A0F6A0BD015502E5C14502F5816
:1007C00011E32F6E306A15502E5E0BD004E21350E9
:1007D000305CF2E007E315502E5E14502F5A135090
:1007E000305AD880113610360F362E362F36303626
:1007F000372EECD70FBE07D00E521DE039320E0651
:10080000372A3936E3D736AC1FD007E215502E5EB3
:1008100014502F5A1350305A17E3113E15D0103E82
:1008200013D00F3E11D00F32103211320E3E0CD0C9
:1008300005D0368604D036840E6A02D036820E6821
:10084000116A106A800E0F6E39AE0F9E11501200A1
:100850000F50306E1318396E0E50D8A412503CE071
:100860000E267E0E03E30E5E03E338D00E5E33E306
:1008700011C02EF010C02FF0308E138E116A106A46
:100880000F6A180E376E30322F322E3206E31550B3
:1008900011261450102213500F220F321032113231
:1008A000372EF1D70FBE07D0113610360F360E5245
:1008B00012E00E06303436AC17D016E3113E14D0D9
:1008C000103E12D00F3E10D0D8800F3210321132AD
:1008D0000E3E0AD003D036840E6A02D036820E68ED
:1008E000116A106A800E0F6E39AE0F9E1150120001
:1008F000106A116A0EC034F011C00EF034C011F04D
:1009000010C034F00FC010F034C00FF0960E376EE8
:10091000396A0EAE07D0D880000E115610560F5609
:100920000E56398E0E5218E036AC0DD011AE0BD0EB
:10093000103E09D00F3E07D00E3E05D0D8800E32B3
:100940000F321032372A080E372610C011F00FC0B0
:1009500010F00EC00FF015D00F6613D0080E375EE2
:10096000105005E1080E375E115011E0116A0F6E4C
:1009700011C010F0116A05D0D890113610360F361C
:1009800037060FAEF9D737C00EF039AE0F9E1150B3
:1009900012003D3D3D3D3D3D3D3D3D3D3D3D3D3DEF
:1009A0003D3D3D3D3D3D3D3D3D3D3D3D3D3D3D3D77
:1009B0003D3D3D3D3D3D3D3D3D004E657720435035
:1009C0005520636869702064657465637465642E7E
:1009D00000003D3D3D3D3D3D3D3D3D3D3D3D3D3DC1
:1009E0003D3D3D3D3D3D3D3D3D3D3D3D3D3D3D3D37
:1009F0003D3D3D3D3D3D3D3D3D003D3D3D3D3D3D64
:100A00003D3D3D3D3D3D3D3D3D3D3D3D3D3D3D3D16
:100A10003D3D3D3D3D3D3D3D3D3D3D3D3D3D3D3D06
:100A20003D0053696572726120526164696F2053A1
:100A3000797374656D732054522053657175656EBA
:100A4000636572004669726D7761726520766572C2
:100A500073696F6E20002C206275696C6420000041
:100A60004E6574776F726B20616464726573732076
:100A70002000456E746572202F2F68656C702066AB
:100A80006F7220636F6D6D616E642073756D6D6143
:100A9000727900003D3D3D3D3D3D3D3D3D3D3D3D8F
:100AA0003D3D3D3D3D3D3D3D3D3D3D3D3D3D3D3D76
:100AB0003D3D3D3D3D3D3D3D3D3D3D00456E74650B
:100AC0007220636F6D6D616E642000004641494C79
:100AD000000048657921206E657720636F6D6D6138
:100AE0006E6400006E65745F7061636B6574207383
:100AF000686F756C6420626520636C656172203C70
:100B000000006E65745F7061636B65745F6C656E29
:100B1000203D20007061636B6574203D20006E6590
:100B2000745F73796E633D006E65745F7479706590
:100B30003D006E65745F66726F6D3D006E65745F3B
:100B4000746F3D006E65745F6372633D00006E6597
:100B5000745F7061796C6F61643D3C006E65745FB9
:100B60007061636B65745F6C656E3D006E65745F8C
:100B70007061796C6F61645F6C656E3D00002E2E54
:100B80002E20636865636B207468652043524320A0
:100B90002E2E2E006C656E677468206F6620617261
:100BA00067203D20000043616C63756C617465646F
:100BB00020435243203D20002C205061636B65741C
:100BC00020435243203D2000435243204661696C3C
:100BD00065642E2020426164207061636B6574003F
:100BE0004352432050617373656420212020476F76
:100BF0006F64205061636B6574006D79206164647B
:100C0000726573733D0048455921207468697320EB
:100C10007061636B657420697320666F72206D6507
:100C200021004E6F74206D79206164647265737366
:100C3000000053656E643A20000053656E643A20EC
:100C4000000053656E643A20000053656E643A20DC
:100C5000000049206861766520746865206E6574BF
:100C6000776F726B20286E65745F61737365727441
:100C7000206163746976652900004E6574776F7230
:100C80006B2072656C656173656400004E6F772040
:100C900061742074686520657865637574655F6E3E
:100CA00065745F636F6D6D616E6420737465700051
:100CB0006E65745F7061636B65745F6C656E3D3DFE
:100CC00000002020636D645F64656C696D3D3D00CC
:100CD0002020636D645F64656C696D3D3D3D00007F
:100CE000636D645F64656C696D20203D0000636D19
:100CF000645F636F6D6D616E643D0000636D645F82
:100D0000617267202020203D00004F4E44454C4139
:100D1000593100004F4E44454C41593200004F4E6E
:100D200044454C41593300004F4E44454C415934E1
:100D300000004F4E44454C41593500004F46464453
:100D4000454C415931004F464644454C41593200CB
:100D50004F464644454C415933004F464644454C66
:100D6000415934004F464644454C41593500454EA3
:100D700041424C45000044495341424C45004E4FCE
:100D8000524D414C4F4E00004F6E2073657175659A
:100D90006E6365203D206E6F726D616C0000524580
:100DA00056455253454F4E004F6E20736571756521
:100DB0006E6365203D2072657665727365004E4FE7
:100DC000524D414C4F4646004F6666207365717523
:100DD000656E6365203D206E6F726D616C005245DB
:100DE00056455253454F464600004F666620736590
:100DF0007175656E6365203D2072657665727365F9
:100E000000004F55543031004F55543032004F558B
:100E1000543033004F55543034004F555430350062
:100E2000494E3100494E3200494E330043570000CD
:100E30004B455945520057504D00574D0000574DF6
:100E40004C494D4954004144314D494E0000414404
:100E5000324D494E00004144334D494E000041445B
:100E6000344D494E00004144314D41580000414449
:100E7000324D415800004144334D41580000414437
:100E8000344D415800004144414C41524D004144D1
:100E900043414C310000414443414C320000414445
:100EA00043414C330000414443414C34000053451E
:100EB0005452455600005345544255494C44000095
:100EC0004E4554004C4F43414C0048454C500000A7
:100ED0004C4F414400005341564500005354415487
:100EE0005553000053544154450044454255474F23
:100EF0004E004465627567206D6F6465204F4E003B
:100F000044454255474F4646000044656275672098
:100F10006D6F6465204F464600005352444542556C
:100F2000474F4E0053686966742072656769737431
:100F30006572206465627567206D6F6465204F4E31
:100F40000000535244454255474F464600005368FF
:100F5000696674207265676973746572206465627E
:100F60007567206D6F6465204F4646004E455444BA
:100F7000454255474F4E00004E6574776F726B20A7
:100F80006465627567206D6F6465204F4E004E4545
:100F90005444454255474F4646004E6574776F723C
:100FA0006B206465627567206D6F6465204F4646EF
:100FB000000050494E470000524F4C4C43414C4CAE
:100FC0000000464F5243454641494C004559454370
:100FD000414E44590000455945004D53474449523C
:100FE00045435400536574206D65737361676520D4
:100FF0006D6F646520746F206469726563742E0080
:101000004D53474E45540000536574206D6573730E
:10101000616765206D6F646520746F206E657477FD
:101020006F726B207061636B6574206D6F64652EE9
:1010300000004543484F0000524553455400524577
:10104000424F4F54000047455441444452005345D9
:101050005441444452005241440053494C454E547B
:1010600000004D4F44450000424F4F5400002050B7
:10107000494E473A20002C2046726F6D3A200000FE
:101080002C20416464726573733A200053544154B8
:1010900045313A005354415445313A005354415478
:1010A00045313A005354415445323A005354415467
:1010B00045333A005354415445343A005354415453
:1010C00045353A005354415445313A005354415444
:1010D00045323A005354415445333A005354415435
:1010E00045343A005354415445353A004F4B0000C3
:1010F00053595354454D204641494C2C2066726F3C
:101100006D3A20002E20205368757474696E672034
:10111000646F776E2E004F4E00004B65796572202C
:101120006D6F6465204F4E004B65796572206D6F61
:101130006465204F46460000536574204357207372
:101140007065656420746F20000053656E642043F1
:10115000573A20002D2D2D2D2D20412F4420434F77
:101160004E5645525445522056414C554553202D1C
:101170002D2D2D2D2D2D2D2D0000416E616C6F67B5
:1011800020696E2031203D200000762020467764C3
:1011900020202800416E616C6F6720696E2032202C
:1011A0003D20000076202052656620202800416EF8
:1011B000616C6F6720696E2033203D20000076202F
:1011C0002020202020202800416E616C6F6720695C
:1011D0006E2034203D20000076202020202020207A
:1011E00028002D2D2D2D2D2D2D2D2D2D2D2D2D2D61
:1011F0002D2D2D2D2D2D2D2D2D2D2D2D2D2D2D2D1F
:101200002D2D2D2D2D2D00004F4E0000416E616CB7
:101210006F6720696E70757420616C61726D206DEE
:101220006F6465204F4E00004F464600416E616C72
:101230006F6720696E70757420616C61726D206DCE
:101240006F6465204F46460053657420412F44204B
:1012500031206D696E696D756D20746F2000536566
:101260007420412F442032206D696E696D756D20A8
:10127000746F200053657420412F442033206D6922
:101280006E696D756D20746F200053657420412F59
:10129000442034206D696E696D756D20746F200077
:1012A00053657420412F442031206D6178696D753C
:1012B0006D20746F200053657420412F442032202C
:1012C0006D6178696D756D20746F200053657420B1
:1012D000412F442033206D6178696D756D20746FE6
:1012E000200053657420412F442034206D617869BB
:1012F0006D756D20746F200053657420412F44205C
:10130000696E70757420312063616C6962726174FA
:10131000696F6E2076616C756520746F200053656F
:101320007420412F4420696E7075742032206361EF
:101330006C6962726174696F6E2076616C7565208C
:10134000746F200053657420412F4420696E7075BE
:101350007420332063616C6962726174696F6E20FE
:1013600076616C756520746F200053657420412F81
:101370004420696E70757420342063616C696272F8
:101380006174696F6E2076616C756520746F2000E2
:10139000212121204C6F7720766F6C746167652066
:1013A000616C61726D206F6E20696E7075742023A0
:1013B000302E20204D696E203D200000762E20200A
:1013C00041637475616C203D2000212121204C6F08
:1013D0007720766F6C7461676520616C61726D2037
:1013E0006F6E20696E7075742023312E20204D6938
:1013F0006E203D200000762E202041637475616CC4
:10140000203D2000212121204C6F7720766F6C74C5
:1014100061676520616C61726D206F6E20696E700E
:1014200075742023322E20204D696E203D2000004F
:10143000762E202041637475616C203D20002121AF
:1014400021204C6F7720766F6C7461676520616C2A
:1014500061726D206F6E20696E7075742023332E5B
:1014600020204D696E203D200000762E2020416313
:101470007475616C203D2000212121204F7665721A
:1014800020766F6C7461676520616C61726D206F8E
:101490006E20696E7075742023302E20204D617887
:1014A000203D2000762E202041637475616C203D24
:1014B0002000212121204F76657220766F6C7461A7
:1014C000676520616C61726D206F6E20696E70754A
:1014D000742023312E20204D6178203D2000762E6F
:1014E000202041637475616C203D20002121212062
:1014F0004F76657220766F6C7461676520616C61F0
:10150000726D206F6E20696E7075742023322E20EC
:10151000204D6178203D2000762E20204163747597
:10152000616C203D2000212121204F7665722076BC
:101530006F6C7461676520616C61726D206F6E20E5
:10154000696E7075742023332E20204D6178203D04
:101550002000762E202041637475616C203D2000B0
:101560004F46460057617474206D65746572207033
:10157000726F74656374696F6E2064697361626C05
:10158000656400004F4E000042617369632077611B
:101590007474206D657465722070726F7465637405
:1015A000696F6E20656E61626C65640043555354CB
:1015B0004F4D0000456E61626C6520757365722049
:1015C000646566696E65642077617474206D657406
:1015D00065722070726F74656374696F6E207261DA
:1015E0006E6765004B657920696E70757420676F52
:1015F000657320696E616374697665004B65792057
:10160000696E70757420676F6573206163746976A5
:10161000650053494C454E540000564552424F53C5
:101620004500426F6F7420696E20766572626F7339
:1016300065206D6F646500004F4E000053696C6556
:101640006E74206D6F6465204F4646004C4F4341D9
:101650004C004E4554574F524B0043616C6C207305
:1016600069676E2073657420746F20005365742061
:101670006669726D776172652072657620746F207D
:101680000000536574206669726D7761726520622F
:1016900075696C6420746F2000004E6574776F72FA
:1016A0006B20616464726573732073657420746F5A
:1016B0002000536574206D79206E6574776F726BAE
:1016C000206164647265737320746F200000536539
:1016D00074205478204F4E2064656C61792031204D
:1016E000746F2000536574205478204F4E20646539
:1016F0006C6179203220746F200053657420547817
:10170000204F4E2064656C6179203320746F200077
:10171000536574205478204F4E2064656C617920A5
:101720003420746F2000536574205478204F4E206D
:1017300064656C6179203520746F200053657420D6
:1017400052782064656C6179203120746F2000002C
:101750005365742052782064656C6179203220745E
:101760006F2000005365742052782064656C6179A5
:10177000203320746F200000536574205278206459
:10178000656C6179203420746F20000053657420EB
:1017900052782064656C6179203520746F200000D8
:1017A0004F7574707574200020656E61626C65649D
:1017B00000004F7574707574200020646973616255
:1017C0006C6564004F4E00004F4646005475726EC3
:1017D000206F75747075742031204F4E0000547561
:1017E000726E206F75747075742031204F464600FC
:1017F0004F4E00004F4646005475726E206F757450
:101800007075742032204F4E00005475726E206F38
:1018100075747075742032204F4646004F4E00009C
:101820004F4646005475726E206F75747075742043
:1018300033204F4E00005475726E206F75747075B2
:10184000742033204F4646004F4E00004F4646005E
:101850005475726E206F75747075742034204F4EFD
:1018600000005475726E206F75747075742034208A
:101870004F4646004F4E00004F4646005475726E6C
:10188000206F75747075742035204F4E00005475AC
:10189000726E206F75747075742035204F46460047
:1018A0004F4E00004F4646005475726E20696E70B0
:1018B00075742031204F4E005475726E20696E7021
:1018C00075742031204F464600004F4E00004F46B1
:1018D00046005475726E20696E7075742032204F08
:1018E0004E005475726E20696E7075742032204FF0
:1018F000464600004F4E00004F4646005475726E3B
:1019000020696E7075742033204F4E005475726ECE
:1019100020696E7075742033204F46460000526572
:1019200073657420616C6C20706172616D657465A3
:10193000727320746F2064656661756C74207661C3
:101940006C7565732E00436F6E666967757261749E
:10195000696F6E20736176656420746F20666C61B8
:101960007368206D656D6F72792E0000436F6E662F
:10197000696775726174696F6E206C6F616465640C
:101980002066726F6D20666C617368206D656D6F87
:1019900072792E002D2D2D20545220537175656EB5
:1019A00063657220436F6D6D616E6473202D2D2D04
:1019B0002D2D2D2D2D2D2D2D2D2D2D2D2D2D2D2D57
:1019C0002D2D2D2D2D2D2D2D2D2D2D2D2D2D2D0074
:1019D0004F4E44454C4159306E207820206D732E77
:1019E0002044656C617920782028312D35303030E5
:1019F00029206D732E206265666F72652074757282
:101A00006E696E67206F6E206F7574707574202319
:101A10006E2C20207768657265206E203D20312D68
:101A200035004F464644454C4159306E2078206D74
:101A3000732E2044656C617920782028312D353053
:101A4000303029206D732E206265666F72652074B8
:101A500075726E696E67206F6666206F757470753B
:101A60007420236E2C207768657265206E203D20DF
:101A7000312D35004E4F524D414C4F4E20202020ED
:101A800020202020205475726E206F6E2020696EF9
:101A9000206E6F726D616C202073657175656E6369
:101AA000652C20312C20322C20332C20342C203556
:101AB00020202844656661756C7429004E4F524D94
:101AC000414C4F4646202020202020202054757273
:101AD0006E206F666620696E206E6F726D616C207D
:101AE0002073657175656E63652C20352C20342C50
:101AF00020332C20322C203120202844656661754B
:101B00006C742900524556455253454F4E202020B3
:101B100020202020205475726E206F6E2020696E68
:101B200020726576657273652073657175656E6385
:101B3000652C20352C20342C20332C20322C2031C5
:101B40000000524556455253454F4646202020201E
:101B50002020205475726E206F666620696E207298
:101B60006576657273652073657175656E63652C46
:101B700020312C20322C20332C20342C2035000016
:101B8000454E41424C452078202020202020202016
:101B900020456E61626C6573206F7574707574207A
:101BA000782028312D35290044495341424C4520A5
:101BB00078202020202020202044697361626C65F9
:101BC00073206F757470757420782028312D352935
:101BD00000002D2D2D2041646D696E20436F6D6DC9
:101BE000616E6473202D2D2D2D2D2D2D2D2D2D2D40
:101BF0002D2D2D2D2D2D2D2D2D2D2D2D2D2D2D2D15
:101C00002D2D2D2D2D2D2D2D2D2D2D2D2D2D00005E
:101C100048454C502020202020202020202020201B
:101C200020446973706C61792074686973206865F9
:101C30006C7020696E666F726D6174696F6E000002
:101C40005354415455532020202020202020202070
:101C500020446973706C61792074686520637572C3
:101C600072656E7420636F6E666967757261746900
:101C70006F6E00004C4F4144202020202020202067
:101C800020202020204C6F616420636F6E6669679E
:101C900075726174696F6E2066726F6D20666C611B
:101CA0007368206D656D6F72790053415645202031
:101CB0002020202020202020202020536176652015
:101CC000636F6E66696775726174696F6E20746F99
:101CD00020666C617368206D656D6F727900524586
:101CE0005345542020202020202020202020205236
:101CF00065736574206F7065726174696E672070BA
:101D00006172616D657465727320746F20737461A4
:101D10006E646172642064656661756C74207661BE
:101D20006C75657300005245424F4F5420202020AF
:101D3000202020202020205265626F6F742074685C
:101D4000652073797374656D0000424F4F542053C2
:101D5000494C454E542020202020205475726E732B
:101D6000206F666620626F6F74206D6573736167A4
:101D70006500424F4F5420564552424F5345202054
:101D80002020205475726E73206F6E20626F6F7406
:101D9000206D65737361676500002D2D2D20412F27
:101DA0004420436F6E766572746572202D20416EFB
:101DB000616C6F6720496E7075742043616C696255
:101DC000726174696F6E2D2D2D2D2D2D2D2D2D2DC4
:101DD0002D2D2D2D2D2D0000414443414C6E20789A
:101DE000787820202020202020416473206F7220EA
:101DF00073756274726163747320746865206F66B2
:101E000066736574207878782028696E206D696C17
:101E100069766F6C74732920746F20746865204133
:101E20002F4420636F6E76657274657220276E276B
:101E3000202028312D34290041446E4D494E207810
:101E400078782020202020202053657473206C6F28
:101E500077207472696767657220616C61726D20AA
:101E6000766F6C7461676520746F2078787820765F
:101E70006F6C74732028696E20766F6C7473290000
:101E800041446E4D41582078787820202020202031
:101E90002053657473206869676820747269676786
:101EA000657220616C61726D20766F6C746167651C
:101EB00020746F2078787820766F6C74732028698E
:101EC0006E20766F6C7473290000524144202020EC
:101ED0002020202020202020202020526561642006
:101EE000616E616C6F6720696E70757420766F6CBF
:101EF00074616765206E6F7700002D2D2D2057616E
:101F00007474204D6574657220436F6D6D616E64ED
:101F100073202D2D2D2D2D2D2D2D2D2D2D2D2D2DB8
:101F20002D2D2D2D2D2D2D2D2D2D2D2D2D2D2D2DE1
:101F30002D2D2D2D2D2D0000574D204F4E202020D2
:101F40002020202020202020205475726E206F6ECB
:101F50002062617369632077617474206D657465B4
:101F600072206D6F6E69746F72696E672E202048E3
:101F7000696768207265666C656374656420706F5C
:101F80007765722064697361626C65732073657133
:101F900075656E6365720000574D204F46462020E0
:101FA0002020202020202020205475726E206F6673
:101FB000662062617369632077617474206D657453
:101FC0006572206D6F6E69746F72696E672E0000A6
:101FD000574D20435553544F4D2020202020202082
:101FE000205475726E206F6E2077617474206D6559
:101FF000746572206D6F6E69746F72696E672E20E2
:1020000020496E68696269742073657175656E63D5
:1020100065207768656E207265666C6563746564BB
:1020200020766F6C746167652068697473207468CA
:102030006520574D4C494D49542076616C756500BB
:10204000574D4C494D495420787878202020202045
:10205000204D696E696D756D207265666C6563747F
:10206000656420766F6C74616765207468617420A4
:1020700077696C6C20696E68696269742074686540
:102080002073657175656E6365002D2D2D20435796
:1020900020436F6D6D616E6473202D2D2D2D2D2DC0
:1020A0002D2D2D2D2D2D2D2D2D2D2D2D2D2D2D2D60
:1020B0002D2D2D2D2D2D2D2D2D2D2D2D2D2D2D2D50
:1020C0002D2D2D2D2D2D00004B45594552204F4EC5
:1020D0002020202020202020205475726E206F6E3A
:1020E000206B65796572206D6F64652E20204F75B9
:1020F0007470757420352077696C6C2073656E641C
:10210000204357207573696E6720746865204357B4
:1021100020636F6D6D616E6400004B455945522020
:102120004F464620202020202020205475726E200B
:102130006F6666206B65796572206D6F64652E2011
:10214000204F757470757420352077696C6C206F22
:1021500070657261746520696E206E6F726D616C5E
:102160002073657175656E636572206D6F646500BF
:10217000435720787878787820202020202020204D
:102180002053656E64207465787420787878787848
:1021900020696E204357207573696E67206F7574D0
:1021A000707574203520696E206B65796572206DBD
:1021B0006F64650057504D20787820202020202023
:1021C00020202020205365742043572073706565BC
:1021D0006420696E20617070726F78696D617465DA
:1021E00020776F72647320706572206D696E7574EC
:1021F000652028312D39392900002D2D2D204E65DF
:1022000074776F726B20436F6D6D616E6473202DF8
:102210002D2D2D2D2D2D2D2D2D2D2D2D2D2D2D2DEE
:102220002D2D2D2D2D2D2D2D2D2D2D2D2D2D2D2DDE
:102230002D2D2D2D2D2D0000534554414444522069
:10224000787820202020202020576865726520782B
:10225000782069732074686520626F6172642773E7
:10226000206E6574776F726B20616464726573733E
:1022700020286265747765656E203120616E642068
:102280003135290047455441444452202020202024
:102290002020202020476574207468652076616CBA
:1022A0007565206F662074686520626F61726427AF
:1022B00073206E6574776F726B20616464726573EE
:1022C000730053494C454E54204F4E20202020206F
:1022D000202020446F206E6F742073656E64206D23
:1022E0006573736167657320746F207365726961CC
:1022F0006C20706F7274207768656E2073746174DF
:1023000065206368616E6765730053494C454E54A0
:10231000204F46462020202020202053656E642038
:102320006D6573736167657320746F20736572697F
:10233000616C20706F7274207768656E20737461B1
:102340007465206368616E67657300004D53474490
:1023500049524543542020202020202020536574DA
:1023600020726573706F6E736520746F20706C617E
:10237000696E207465787420666F726D61740000F8
:102380004D53474E4554202020202020202020203F
:102390002053657420726573706F6E736520746F5F
:1023A000206E6574776F726B207061636B6574204B
:1023B000666F726D617400002D2D2D204D616E755C
:1023C000616C204F757470757420436F6D6D616E14
:1023D0006473202D2D2D2D2D2D2D2D2D2D2D2D2DBD
:1023E0002D2D2D2D2D2D2D2D2D2D2D2D2D2D2D2D1D
:1023F0002D2D2D2D00004F5554306E204F4E202096
:10240000202020202020204D616E75616C6C792089
:102410007475726E204F4E20206F75747075742025
:102420006E2028312D3529004F5554306E204F46EF
:102430004620202020202020204D616E75616C6C8C
:1024400079207475726E204F4646206F75747075D2
:1024500074206E2028312D3529002D2D2D20496E18
:102460007465726E616C20446562756767696E673A
:1024700020436F6D6D616E6473202D2D2D2D2D2DDC
:102480002D2D2D2D2D2D2D2D2D2D2D2D2D2D2D2D7C
:102490002D2D2D2D2D2D000044454255474F4E200A
:1024A0002020202020202020205475726E206F6E66
:1024B00020646562756767696E67206D6573736117
:1024C0006765730044454255474F4646202020200B
:1024D00020202020205475726E206F66662064656F
:1024E00062756767696E67206D6573736167657391
:1024F0000000464F5243454641494C2020202020B1
:10250000202020466F7263657320756E69742069A0
:102510006E746F204641494C206D6F64652E2020FB
:102520005368757473206F666620616C6C206F75DC
:102530007470757473003D3D3D3D3D5B20435552C5
:1025400052454E5420434F4E4649475552415449F7
:102550004F4E205D3D3D3D3D3D3D3D3D3D00436F8A
:102560006E66696720636F646520203A2000426FC1
:1025700061726420747970652020203A20004657EB
:102580002076657273696F6E2020203A20004657CE
:10259000206275696C6420202020203A20004D794B
:1025A00020616464726573732020203A20004F4ECE
:1025B000202064656C6179203120203A20004F4E44
:1025C000202064656C6179203220203A20004F4E33
:1025D000202064656C6179203320203A20004F4E22
:1025E000202064656C6179203420203A20004F4E11
:1025F000202064656C6179203520203A20004F4608
:10260000462064656C6179203120203A20004F46D5
:10261000462064656C6179203220203A20004F46C4
:10262000462064656C6179203320203A20004F46B3
:10263000462064656C6179203420203A20004F46A2
:10264000462064656C6179203520203A20003A20CC
:10265000456E61626C6564003A2044495341424CC6
:10266000454400004F75747075742031202020207F
:1026700020003A20456E61626C6564003A2044494E
:102680005341424C454400004F75747075742032BC
:102690002020202020003A20456E61626C65640095
:1026A0003A2044495341424C454400004F757470F0
:1026B000757420332020202020003A20456E61626E
:1026C0006C6564003A2044495341424C4544000043
:1026D0004F757470757420342020202020003A201B
:1026E000456E61626C6564003A2044495341424C36
:1026F000454400004F7574707574203520202020EB
:1027000020004F4E2073657175656E636520203A19
:10271000204E6F726D616C004F4E20736571756550
:102720006E636520203A2052657665727365640099
:102730004F46462073657175656E6365203A204E7D
:102740006F726D616C004F46462073657175656EE2
:102750006365203A2052657665727365640043575D
:1027600020737065656420202020203A2000576186
:102770007474206D6574657220636865636B696E3F
:1027800067204F46460053696D706C652077617411
:1027900074206D6574657220636865636B696E672C
:1027A00020656E61626C6564000057617474206D11
:1027B00065746572206C696D69742073657420742A
:1027C0006F200000414420616C61726D206D6F6468
:1027D000653A204F66660000414420616C61726D6D
:1027E000206D6F64653A204F4E00416E616C6F67DB
:1027F0002031206D696E203A2000202020202020EA
:102800002020206D6178203A2000202020202020E8
:1028100020202063616C203A2000416E616C6F675C
:102820002032206D696E203A2000202020202020B8
:102830002020206D6178203A2000202020202020B8
:1028400020202063616C203A2000416E616C6F672C
:102850002033206D696E203A200020202020202087
:102860002020206D6178203A200020202020202088
:1028700020202063616C203A2000416E616C6F67FC
:102880002034206D696E203A200020202020202056
:102890002020206D6178203A200020202020202058
:1028A00020202063616C203A2000436F6D6D206D05
:1028B0006F6465202020203A204C6F63616C00001B
:1028C000436F6D6D206D6F6465202020203A204E8F
:1028D0006574776F726B0000F86A400E366E006A9E
:1028E000030EAF6E200EAC6E900EAB6E2EEE81F02E
:1028F00094988298949A829A9390819093928192DC
:1029000093948194110E05012C6FC70E2B6F510EFD
:102910002A6F810E296F0101D79DD78F040E176E84
:10292000B00E166E1B6A8EC51AF044EC02F005015B
:102930008C6F17C08DF5030E8B6F520E8A6F05EEEC
:10294000DAF0540EEE6E520EEE6E310EEE6EEF6A4F
:102950000001E2EF14F09EAA23D0060EAB141DE195
:10296000E2CF3BF0E1CF3AF03C2AFF0E3C5C01E3C2
:102970003C6A1DEE82F03C50E126000EE222AECF12
:10298000E7FF0D0EE75C02E1010E406E3CC015F45E
:102990003BC0E2FF3AC0E1FF1100AB98AB8800D02A
:1029A00011003C6A3D6A9D8AC00EF26E12009D9A2B
:1029B0000DEE82F0FF0EEE6AE82EFDD73C6A3D6A0E
:1029C0009D8A1200400EAF6E900EAB6E200EAC6E64
:1029D0000B0EC16EF19E320ECCEC01F08298829A01
:1029E0008190819281949394819493928192939017
:1029F0008190949A829A949882980101D79BD7BF2C
:102A00008282D7AF8292050128910101CA6BD26BF5
:102A1000D96BD86B01EEDAF04F0EEE6E4B0EEE6E08
:102A2000EF6A01EE1AF0EE6A01EEDFF0EE6A0401E1
:102A30009E6B640E9D6FA06B9F6B04EE17F0300EC3
:102A4000EE6EEE6EEF6A06010589058B059D0401A9
:102A5000A16B04EEA2F0EE6A0501256B246BE489FC
:102A6000E48BE48DE48F0601058105930501756B08
:102A7000CD0E796FCC0E786F4C0E776F7C0E766F23
:102A80000601059505970101666B686B0501236BCF
:102A9000486B476B466B456B4C6B4B6B4A6B496B9A
:102AA000506B4F6B4E6B4D6B546B536B526B516B4A
:102AB0000101696B0501586B576B566B556B5C6B6D
:102AC0005B6B5A6B596B606B5F6B5E6B5D6B646BC2
:102AD000636B626B616B686B676B700E666F830E06
:102AE000656F6C6B6B6B700E6A6F830E696F706BCA
:102AF0006F6B700E6E6F830E6D6F746B736B700EF9
:102B0000726F830E716F01016A6B4BDF000184EC01
:102B100017F00101D791D793D795010E0501E16F09
:102B2000010ED56FD76B040ED66FD96B1E0ED86F02
:102B3000010EE36F586B576B566B556B686B676B89
:102B4000200E666F810E656F5C6B5B6B5A6B596B09
:102B50006C6B6B6B200E6A6F810E696F606B5F6BC5
:102B60005E6B5D6B706B6F6B200E6E6F810E6D6FA9
:102B7000646B636B626B616B746B736B200E726F53
:102B8000810E716FE497276B640E266FE129E26F67
:102B90000001F4EC28F082B6CFEF15F0F9D794904D
:102BA0008280000E9DEC01F00501D56FD529000152
:102BB000D8A406EF16F00401A1530001D8A406EF33
:102BC00016F004EEA2F0090EF76E920EF66E81EC8E
:102BD00002F0EF6A65EC1DF004EEA2F0090EF76E4C
:102BE000BA0EF66E81EC02F0EF6A65EC1DF026EC91
:102BF00040F0C1EC40F004EEA2F0090EF76ED20EE8
:102C0000F66E81EC02F0EF6A65EC1DF0D4EC43F057
:102C10000BEC37F001EE6BF0020E016E0501E35193
:102C2000CCEC00F0EF6A010E0401A153D8A4000E11
:102C3000336E010E01016953D8A4000E3314000154
:102C4000D8B48DEF16F004EEA2F0090EF76EFA0E6E
:102C5000F66E81EC02F0EF6A65EC1DF004EEA2F076
:102C60000A0EF76E220EF66E81EC02F0EF6A65EC4A
:102C70001DF004EEA2F00A0EF76E440EF66E81EC23
:102C800002F0020E016E066AD7C51FF0D6C51EF00F
:102C9000CFEC00F00A0EF76E560EF66E81EC02F0E5
:102CA000020E016E066AD9C51FF0D8C51EF0CFEC22
:102CB00000F0EF6A65EC1DF004EEA2F00A0EF76E6C
:102CC000600EF66E81EC02F0020E016E0501E3511A
:102CD000CCEC00F0EF6A04EEA2F00A0EF76E720E72
:102CE000F66E81EC02F0EF6A000165EC1DF004EE77
:102CF000A2F00A0EF76E940EF66E81EC02F0EF6A07
:102D000065EC1DF004EEA2F00A0EF76EBC0EF66E36
:102D100081EC02F0EF6A65EC1DF0320ECCEC01F0B4
:102D2000949082900A0EF76ECC0EF66E01EEDAF0F9
:102D3000A9EC02F0D8A49FEF16F055EC29F0D89634
:102D4000060105ADD8860001D8B6A9EF16F0DEEF72
:102D500016F001EE9EF0020E016EE86A80BA010ED6
:102D6000CCEC00F0EF6A01EE9EF084EC00F0808A7B
:102D7000E8A0809A01EEB3F0020E016EE86A81B617
:102D8000010ECCEC00F0EF6A01EEB3F084EC00F041
:102D90008186E8A081962DEC2EF0010E01016A5D7E
:102DA0000001D8A4D6EF16F0EFEC33F0050175530F
:102DB0000001D8B4DEEF16F096EC36F00601059D62
:102DC000000181A8E6EF16F044EF17F0010E0101B3
:102DD000CA6FE86A80BA010E336EE86A81B6010EE6
:102DE00033100001D8B4FAEF16F00101CA6B0001EC
:102DF000FDEF16F0010E0101CA6F0001010E010185
:102E0000CA5D010ED8A4000E336E010E050128BD67
:102E1000E86A33140001D8B410EF17F0DEEF3AF08F
:102E2000010E0101CA5D010ED8A4000E336EE86ADE
:102E3000050128BD010E33140001D8B422EF17F0AC
:102E40001CEF37F0010E0101CA53D8A4000E336EF7
:102E5000010E050128BDE86A33140001D8B433EF30
:102E600017F0F8EF38F0010E0101CA53D8A4000E94
:102E7000336EE86A050128BD010E33140001D8B491
:102E800044EF17F0E3EF3AF00501244B252B2451D2
:102E9000265D255127590001D8B06DEF17F00501C7
:102EA000256B246BD89628B1D8860001D8B660EF80
:102EB00017F0050128819492829200016DEF17F0BE
:102EC000D896050128A1D8860001D8B66CEF17F076
:102ED0000501289194928282000104019F519D5D19
:102EE000A0519E590001D8B07BEF17F084EC17F089
:102EF0000401A06B9F6B0001010E405CD8A483EF1E
:102F000017F088EC17F00ED7406AD7EC14F01200D7
:102F1000D8960101D7A5D8860001D8B69CEF17F046
:102F20000A0EF76ED20EF66E82EC01F00D0E8AECF0
:102F300001F00A0E8AEC01F001EEDFF0820EEE6A7B
:102F4000E82EFDD7D8960101D7A5D8860001D8B6BE
:102F5000C0EF17F00A0EF76EE40EF66E82EC01F089
:102F600001EEDFF0EE5003E08AEC01F0FBD73E0EFD
:102F70008AEC01F00D0E8AEC01F00A0E8AEC01F0E9
:102F80003C040401156F00013CAEC9EF17F00401C9
:102F9000156B0001D8960101D7A5D8860001D8B6D7
:102FA000E4EF17F00B0EF76E020EF66E82EC01F0F6
:102FB000040E016E04011551CCEC00F00D0E8AECEC
:102FC00001F00A0E8AEC01F0000104011553000122
:102FD000D8A4EEEF17F0010E0401156F00010401F3
:102FE0001505096E0101CA6B00010101CA51095C96
:102FF0000001D8A034EF18F0D8960101CAAFD886E6
:103000000001D8B606EF18F00101CA6B00010101FA
:10301000CA290DEE82F0E926000EEA22EFCF0DF06C
:1030200001EEDFF0CA51E926000EEA220DC0EFFFE3
:10303000D896D7A5D8860001D8B62EEF18F0040E82
:10304000016E01EEDFF00101CA51E926000EEA220D
:10305000EF50CCEC00F0200E8AEC01F000010101F1
:10306000CA2B0001D8A4C0D737EC18F0120001EE2B
:10307000DFF011EEDFF09DEC02F0D8960101D7A54C
:10308000D8860001D8B658EF18F00B0EF76E140E64
:10309000F66E82EC01F001EEDFF0EE5003E08AEC18
:1030A00001F0FBD70D0E8AEC01F00A0E8AEC01F05C
:1030B00002EE61F011EEDFF0010EF36E010E89EC0D
:1030C00002F0EF6AD8960101D7A5D8860001D8B6DC
:1030D0007DEF18F00B0EF76E1E0EF66E82EC01F00F
:1030E00002EE61F0EE5003E08AEC01F0FBD70D0E2A
:1030F0008AEC01F00A0E8AEC01F002EE63F011EEA8
:10310000DFF0020EF36E010E89EC02F0EF6AD89642
:103110000101D7A5D8860001D8B6A2EF18F00B0E92
:10312000F76E280EF66E82EC01F002EE63F0EE50C0
:1031300003E08AEC01F0FBD70D0E8AEC01F00A0ED9
:103140008AEC01F002EE66F011EEDFF0030EF36E92
:10315000020E89EC02F0EF6AD8960101D7A5D88655
:103160000001D8B6C7EF18F00B0EF76E320EF66EF0
:1031700082EC01F002EE66F0EE5003E08AEC01F022
:10318000FBD70D0E8AEC01F00A0E8AEC01F002EE7C
:103190006AF011EEDFF0050EF36E020E89EC02F01C
:1031A000EF6AD8960101D7A5D8860001D8B6ECEF12
:1031B00018F00B0EF76E3C0EF66E82EC01F002EE8C
:1031C0006AF0EE5003E08AEC01F0FBD70D0E8AECBA
:1031D00001F00A0E8AEC01F002EE6EF011EEDFF063
:1031E000070EF36E030E89EC02F0EF6AD896010128
:1031F000D7A5D8860001D8B611EF19F00B0EF76EDF
:10320000440EF66E82EC01F002EE6EF0EE5003E03A
:103210008AEC01F0FBD70D0E8AEC01F00A0E8AEC65
:1032200001F002EE73F011EEDFF00A0EF36E090EFC
:103230000401155D89EC02F0EF6AD8960101D7A56B
:10324000D8860001D8B63BEF19F00B0EF76E4E0E84
:10325000F66E82EC01F002EE73F0EE5003E08AECC1
:1032600001F0FBD73E0E8AEC01F00D0E8AEC01F066
:103270000A0E8AEC01F001EEDFF0E86AEE5202E09D
:10328000E83EFCD70401156FD8960101D7A5D88672
:103290000001D8B65EEF19F00B0EF76E5C0EF66EFD
:1032A00082EC01F0040E016E04011551CCEC00F02B
:1032B0000D0E8AEC01F00A0E8AEC01F0000102EE1C
:1032C00073F0E86AEE5202E0E83EFCD70401166FA4
:1032D000D8960101D7A5D8860001D8B682EF19F09B
:1032E0000B0EF76E6C0EF66E82EC01F0040E016EA2
:1032F00004011651CCEC00F00D0E8AEC01F00A0E20
:103300008AEC01F0000104EE17F012EE66F0030EF5
:10331000E75204E0E6CFEEFFE82EFAD7EF6A300E70
:103320000201635D0001D8A498EF19F03CEF1BF097
:103330002F0E0201635D0001D8A4A1EF19F0010175
:10334000D78B00012F0E0201635D0001D8A4AEEF00
:1033500019F004EE17F0300EEE6EEF6A2F0E020138
:10336000635D0001D8A4B7EF19F0EFEC1EF02F0E4B
:103370000201635D0001D8A4C3EF19F00101686B7D
:103380000001C6EF19F0010E0101686F00012F0E58
:103390000201635D0001D8A4CFEF19F01200D896A6
:1033A0000101D7A5D8860001D8B6E3EF19F00B0EBE
:1033B000F76E7E0EF66E82EC01F00D0E8AEC01F0D7
:1033C0000A0E8AEC01F0D8960101D7A5D886000133
:1033D000D8B6FDEF19F00B0EF76E940EF66E82EC78
:1033E00001F0040E016E0101D251CCEC00F00D0E83
:1033F0008AEC01F00A0E8AEC01F000010401146B62
:10340000010E0101CA6F0001060E0101CA5D000133
:10341000D8B067EF1AF001EEDFF00101CA51E926DA
:10342000000EEA22EF50D26FD2510401141B01EEBC
:103430009EF0020E016E0101CA51CCEC00F0EF6A61
:1034400001EEB3F0020E016E04011451CCEC00F059
:10345000EF6AD8960101D7A5D8860001D8B661EFEA
:103460001AF001EE9EF0EE5003E08AEC01F0FBD77B
:10347000200E8AEC01F001EEDFF00101CA51E926CD
:10348000000EEA22EF508AEC01F0200E8AEC01F0E7
:10349000630E8AEC01F0720E8AEC01F0630E8AEC86
:1034A00001F03D0E8AEC01F001EEB3F0EE5003E0C6
:1034B0008AEC01F0FBD70D0E8AEC01F00A0E8AECC3
:1034C00001F000010101CA2B0001D8A49CD7090E0C
:1034D0000101CA6F00010101CA510401155D00011B
:1034E000D8A0CFEF1AF001EEDFF00101CA51E926B2
:1034F000000EEA22EF50096E09500401141B01EE80
:103500009EF0020E016E0101CA51CCEC00F0EF6A90
:1035100001EEB3F0020E016E04011451CCEC00F088
:10352000EF6AD8960101D7A5D8860001D8B6C9EFB1
:103530001AF001EE9EF0EE5003E08AEC01F0FBD7AA
:10354000200E8AEC01F001EEDFF00101CA51E926FC
:10355000000EEA22EF508AEC01F0200E8AEC01F016
:10356000630E8AEC01F0720E8AEC01F0630E8AECB5
:1035700001F03D0E8AEC01F001EEB3F0EE5003E0F5
:103580008AEC01F0FBD70D0E8AEC01F00A0E8AECF2
:1035900001F000010101CA2B0001D8A49BD7D896E5
:1035A0000101D7A5D8860001D8B6F6EF1AF00B0EA8
:1035B000F76EA60EF66E82EC01F0040E016E0401A9
:1035C0001451CCEC00F00B0EF76EB80EF66E82ECD8
:1035D00001F002EE6EF0EE5003E08AEC01F0FBD752
:1035E0000D0E8AEC01F00A0E8AEC01F0000102EEE9
:1035F0006EF084EC00F0096E1FC00AF020C00BF0E2
:1036000021C00CF00B500C100AE10A500B1007E11E
:103610000950040114190001D8B428EF1BF0D89602
:103620000101D7A5D8860001D8B623EF1BF00B0EF9
:10363000F76EC80EF66E82EC01F00D0E8AEC01F00A
:103640000A0E8AEC01F084EC17F012003CEF1BF03C
:10365000D8960101D7A5D8860001D8B63CEF1BF05B
:103660000B0EF76EE00EF66E82EC01F00D0E8AEC9A
:1036700001F00A0E8AEC01F0D8960101D7A5D88690
:103680000001D8B656EF1BF00B0EF76EFA0EF66E71
:1036900082EC01F0040E016E0501E351CCEC00F068
:1036A0000D0E8AEC01F00A0E8AEC01F0000102EE28
:1036B0006AF084EC00F00101D26FD56BD2510501A4
:1036C000E35D0001D8A468EF1BF0010E0101D56F86
:1036D0000001630E0101D25D0001D8A473EF1BF05D
:1036E000010E0101D56F0001630E0101D25D0001E1
:1036F000D8A47EEF1BF0020E0101686F0001010EDD
:103700000101D55D0001D8A4A4EF1BF0D8960101FA
:10371000D7A5D8860001D8B69AEF1BF00C0EF76E2D
:10372000060EF66E82EC01F00D0E8AEC01F00A0E28
:103730008AEC01F002EE73F012EE73F09DEC02F0F1
:1037400006EC1FF0B8EF1BF0D8960101D7A5D8867C
:103750000001D8B6B8EF1BF00C0EF76E220EF66E15
:1037600082EC01F00D0E8AEC01F00A0E8AEC01F0F9
:1037700084EC17F0120002EEC8F011EE2FF0360EB6
:10378000E75204E0E6CFEEFFE82EFAD7EF6ACCEC82
:103790001BF05AEC1EF0120003EE0AF0820EEE6AE5
:1037A000E82EFDD702EEB5F02F0EEE6EEF6A02EEB8
:1037B000B8F0410EEE6EEF6A02EEBBF0020E016E43
:1037C0000501E351CCEC00F0EF6A02EEBBF0E86AD1
:1037D000EE5202E0E83EFCD7096E010E095C0001E2
:1037E000D8A403EF1CF001EEB3F0300EEE6E12EE33
:1037F000BBF0030EE75204E0E6CFEEFFE82EFAD767
:10380000EF6A0FEF1CF001EEB3F012EEBBF0030E07
:10381000E75204E0E6CFEEFFE82EFAD7EF6A02EEB9
:10382000BBF011EEB3F0140EE75204E0E6CFEEFF6A
:10383000E82EFAD7EF6A02EEBFF014EE17F0030E8F
:10384000E75204E0E6CFEEFFE82EFAD7EF6A02EE89
:10385000BFF0E86AEE5202E0E83EFCD70101D26F09
:10386000D2530001D8A43BEF1CF002EEBFF0300EA3
:10387000EE6EEE6EEF6A010E0101D25D0001D8A47A
:103880005CEF1CF004EEA2F0300EEE6E12EEBFF014
:10389000030EE75204E0E6CFEEFFE82EFAD7EF6A18
:1038A00002EEBFF014EEA2F0800EE75204E0E6CF85
:1038B000EEFFE82EFAD7EF6A020E0101D25D000199
:1038C000D8A469EF1CF002EEBFF0EE50FEE1ED521D
:1038D000EF6A01EE6BF012EEB5F0020EE75204E073
:1038E000E6CFEEFFE82EFAD712EEB8F0020EE7525E
:1038F00004E0E6CFEEFFE82EFAD712EEBBF0030E9F
:10390000E75204E0E6CFEEFFE82EFAD712EEBFF062
:10391000030EE75204E0E6CFEEFFE82EFAD712EEF0
:10392000C8F0410EE75204E0E6CFEEFFE82EFAD7EA
:10393000EF6A01EE6BF0E86AEE5202E0E83EFCD777
:103940000101D66FD56B01EE6BF0E86AEE5202E032
:10395000E83EFCD7096E010ECA6F00010101CA5191
:10396000095C0001D8A0D1EF1CF001EE6BF0010161
:10397000CA51EB50D26FD251D51B01EE9EF0020E10
:10398000016ECA51CCEC00F0EF6A01EEB3F0020E0A
:10399000016ED551CCEC00F0EF6ACA2B0001D8A41F
:1039A000DCD702EEC3F0020E016E0101D551CCEC62
:1039B00000F0EF6A02EEC3F0E86AEE5202E0E83E81
:1039C000FCD7D26F010ED25D0001D8A4F7EF1CF036
:1039D00004EEA2F0300EEE6EEE6E12EEC3F0040EA8
:1039E000E75204E0E6CFEEFFE82EFAD7EF6A020EC8
:1039F0000101D25D0001D8A40CEF1DF004EEA2F08D
:103A0000300EEE6E12EEC3F0040EE75204E0E6CF85
:103A1000EEFFE82EFAD7EF6A030E0101D25D000136
:103A2000D8A41FEF1DF004EEA2F012EEC3F0040EB6
:103A3000E75204E0E6CFEEFFE82EFAD7EF6A02EE97
:103A4000C3F014EEA2F0800EE75204E0E6CFEEFFE2
:103A5000E82EFAD7EF6A03EE0AF012EEB5F0020E86
:103A6000E75204E0E6CFEEFFE82EFAD712EEB8F008
:103A7000020EE75204E0E6CFEEFFE82EFAD712EE90
:103A8000BBF0030EE75204E0E6CFEEFFE82EFAD7D4
:103A900012EEBFF0030EE75204E0E6CFEEFFE82E91
:103AA000FAD712EEC3F0040EE75204E0E6CFEEFFC1
:103AB000E82EFAD712EEC8F0410EE75204E0E6CF46
:103AC000EEFFE82EFAD7EF6A1200010168530001F9
:103AD000D8A4B3EF1DF08FEC1EF0D8960101D7A546
:103AE000D8860001D8B688EF1DF00C0EF76E320EA6
:103AF000F66E82EC01F004EEA2F0EE5003E08AECE8
:103B000001F0FBD70D0E8AEC01F00A0E8AEC01F0F1
:103B10000401A1530001D8A49BEF1DF004EEA2F014
:103B2000EE5003E08AEC01F0FBD70D0E8AEC01F0B9
:103B30000A0E8AEC01F0010E0401A15D0001D8A477
:103B4000AFEF1DF004EEA2F0EE5003E08AEC01F0BE
:103B5000FBD70D0E8AEC01F00A0E8AEC01F0D8ECCE
:103B60001EF059EF1EF0010E0101685D0001D8A49E
:103B700002EF1EF08FEC1EF0D8960101D7A5D88673
:103B80000001D8B6D7EF1DF00C0EF76E3A0EF66EA8
:103B900082EC01F004EEA2F0EE5003E08AEC01F0BA
:103BA000FBD70D0E8AEC01F00A0E8AEC01F004013D
:103BB000A1530001D8A4EAEF1DF004EEA2F0EE50EC
:103BC00003E08AEC01F0FBD70D0E8AEC01F00A0E3F
:103BD0008AEC01F0010E0401A15D0001D8A4FEEF02
:103BE0001DF004EEA2F0EE5003E08AEC01F0FBD7EA
:103BF0000D0E8AEC01F00A0E8AEC01F0D8EC1EF0F2
:103C000059EF1EF0020E0101685D0001D8A459EFC2
:103C10001EF00501E351320DF3CF1AF0F4CF1BF083
:103C2000CEEC01F000018FEC1EF0D8960101D7A573
:103C3000D8860001D8B630EF1EF00C0EF76E420E9B
:103C4000F66E82EC01F004EEA2F0EE5003E08AEC96
:103C500001F0FBD70D0E8AEC01F00A0E8AEC01F0A0
:103C60000401A1530001D8A443EF1EF004EEA2F01A
:103C7000EE5003E08AEC01F0FBD70D0E8AEC01F068
:103C80000A0E8AEC01F0010E0401A15D0001D8A426
:103C900057EF1EF004EEA2F0EE5003E08AEC01F0C4
:103CA000FBD70D0E8AEC01F00A0E8AEC01F0D8EC7D
:103CB0001EF012008FEC1EF0D8960101D7A5D88611
:103CC0000001D8B677EF1EF00C0EF76E4A0EF66EB6
:103CD00082EC01F003EE0AF0EE5003E08AEC01F012
:103CE000FBD70D0E8AEC01F00A0E8AEC01F0D89693
:103CF000060105B7D8860001D8B68CEF1EF003EE9A
:103D00000AF0EE5003E08AEC01F0FBD70D0E8AECCE
:103D100001F00A0E8AEC01F0D8EC1EF0120001014D
:103D2000D56B000101EE9EF0020E016EE86A82B6CC
:103D3000010ECCEC00F0EF6A01EE9EF084EC00F096
:103D40000101D26F010ED25D0001D8A4AAEF1EF0CE
:103D5000BEEF1EF00101D52B0501E3510A0DF3CF93
:103D60001AF0F4CF1BF0CEEC01F0330E0101D55D5B
:103D70000001D8A0BDEF1EF01200D3D7949082802E
:103D8000050ECCEC01F0D8960101D7A5D88600012C
:103D9000D8B6D7EF1EF00C0EF76E520EF66E82EC10
:103DA00001F00D0E8AEC01F00A0E8AEC01F012000F
:103DB00094908290D8960101D7A5D8860001D8B6F4
:103DC000EEEF1EF00C0EF76E7A0EF66E82EC01F03E
:103DD0000D0E8AEC01F00A0E8AEC01F01200D89662
:103DE0000101D7ABD8860001D8B605EF1FF002EE6F
:103DF00073F011EEDFF0030EF36E000E0401155D9B
:103E000089EC02F0EF6A0101D79B0001D89601010D
:103E1000D7A5D8860001D8B61AEF1FF00C0EF76EA2
:103E20008C0EF66E82EC01F00D0E8AEC01F00A0E9B
:103E30008AEC01F001EEDFF012EE73F0410EE75272
:103E400004E0E6CFEEFFE82EFAD7EF6A3F6A01EE14
:103E5000DFF0E86AEE5202E0E83EFCD70401156F9D
:103E60000101CA6B00010101CA510401155D000185
:103E7000D8A0BEEF1FF0D8960101D7A5D8860001C3
:103E8000D8B655EF1FF00C0EF76EB00EF66E82EC42
:103E900001F0040E016E04011551CCEC00F00D0E82
:103EA0008AEC01F00A0E8AEC01F00001D8960101BB
:103EB000D7A5D8860001D8B67BEF1FF0690E8AEC33
:103EC00001F03D0E8AEC01F08AEC01F0040E016E67
:103ED0000101CA51CCEC00F00C0EF76EC20EF66E6A
:103EE00082EC01F03F50CCEC00F00D0E8AEC01F0BA
:103EF0000A0E8AEC01F0000101EEDFF00101CA5167
:103F0000E926000EEA22EF50096E200E095C00013E
:103F1000D8A491EF1FF00101CA293F6E0001BEEF46
:103F20001FF0D8960101D7A5D8860001D8B6B8EF02
:103F30001FF0690E8AEC01F03D0E8AEC01F08AEC6C
:103F400001F08AEC01F0040E016E0101CA51CCECC3
:103F500000F00C0EF76ED00EF66E82EC01F03F50C2
:103F6000CCEC00F00D0E8AEC01F00A0E8AEC01F0A8
:103F700000010101CA2B0001D8A474D700EE41F062
:103F800011EEDFF03F04E6CFEEFFE82EFCD7EF6A3C
:103F900000EE41F010EE41F09DEC02F000EE56F024
:103FA00011EEDFF03F500401155D92EC02F0EF6A74
:103FB0003F520001D8A4E0EF1FF000EE56F0EE6A89
:103FC00000EE56F010EE56F09DEC02F001EE2FF0F0
:103FD00010EE56F0400EE75204E0E6CFEEFFE82E7A
:103FE000FAD7EF6AD8960101D7A5D8860001D8B6CE
:103FF0000BEF20F00C0EF76EE00EF66E82EC01F087
:10400000040E016E3F50CCEC00F00D0E8AEC01F076
:104010000A0E8AEC01F0D8960101D7A5D8860001D6
:10402000D8B626EF20F00C0EF76EEE0EF66E82EC90
:1040300001F000EE41F0EE5003E08AEC01F0FBD716
:104040000D0E8AEC01F00A0E8AEC01F0D8960101FF
:10405000D7A5D8860001D8B641EF20F00C0EF76E38
:10406000FC0EF66E82EC01F000EE56F0EE5003E02E
:104070008AEC01F0FBD70D0E8AEC01F00A0E8AECF7
:1040800001F00D0EF76E0A0EF66E00EE41F0A9EC8F
:1040900002F0D8A450EF20F000EC3CF017EF25F030
:1040A0000D0EF76E140EF66E00EE41F0A9EC02F064
:1040B000D8A45FEF20F026EC3CF017EF25F00D0EB2
:1040C000F76E1E0EF66E00EE41F0A9EC02F0D8A4D9
:1040D0006EEF20F04CEC3CF017EF25F00D0EF76E74
:1040E000280EF66E00EE41F0A9EC02F0D8A47DEFA8
:1040F00020F072EC3CF017EF25F00D0EF76E320E4B
:10410000F66E00EE41F0A9EC02F0D8A48CEF20F09E
:1041100098EC3CF017EF25F00D0EF76E3C0EF66EA6
:1041200000EE41F0A9EC02F0D8A49BEF20F0BEEC29
:104130003CF017EF25F00D0EF76E460EF66E00EE12
:1041400041F0A9EC02F0D8A4AAEF20F0E4EC3CF096
:1041500017EF25F00D0EF76E500EF66E00EE41F0E3
:10416000A9EC02F0D8A4B9EF20F00AEC3DF017EF6B
:1041700025F00D0EF76E5A0EF66E00EE41F0A9EC2A
:1041800002F0D8A4C8EF20F030EC3DF017EF25F096
:104190000D0EF76E640EF66E00EE41F0A9EC02F023
:1041A000D8A4D7EF20F056EC3DF017EF25F00D0E18
:1041B000F76E6E0EF66E00EE41F0A9EC02F0D8A498
:1041C000E6EF20F07CEC3DF017EF25F00D0EF76EDA
:1041D000760EF66E00EE41F0A9EC02F0D8A4F5EFF1
:1041E00020F0E2EC3DF017EF25F00D0EF76E7E0E9D
:1041F000F66E00EE41F0A9EC02F0D8A410EF21F029
:104200000601058904EEA2F00D0EF76E880EF66E1B
:1042100081EC02F0EF6A000165EC1DF017EF25F06C
:104220000D0EF76E9E0EF66E00EE41F0A9EC02F058
:10423000D8A42BEF21F00601059904EEA2F00D0E93
:10424000F76EA80EF66E81EC02F0EF6A000165ECE5
:104250001DF017EF25F00D0EF76EBE0EF66E00EE98
:1042600041F0A9EC02F0D8A446EF21F00601058B3D
:1042700004EEA2F00D0EF76EC80EF66E81EC02F0A1
:10428000EF6A000165EC1DF017EF25F00D0EF76EDB
:10429000DE0EF66E00EE41F0A9EC02F0D8A461EF5C
:1042A00021F00601059B04EEA2F00D0EF76EEA0E5A
:1042B000F66E81EC02F0EF6A000165EC1DF017EF7D
:1042C00025F00E0EF76E020EF66E00EE41F0A9EC30
:1042D00002F0D8A470EF21F048EC3EF017EF25F083
:1042E0000E0EF76E080EF66E00EE41F0A9EC02F02D
:1042F000D8A47FEF21F07DEC3EF017EF25F00E0EF5
:10430000F76E0E0EF66E00EE41F0A9EC02F0D8A4A6
:104310008EEF21F0B2EC3EF017EF25F00E0EF76EA7
:10432000140EF66E00EE41F0A9EC02F0D8A49DEF59
:1043300021F0E7EC3EF017EF25F00E0EF76E1A0EA7
:10434000F66E00EE41F0A9EC02F0D8A4ACEF21F03B
:104350001CEC3FF017EF25F00E0EF76E200EF66EF8
:1043600000EE41F0A9EC02F0D8A4BBEF21F054EC30
:104370003FF017EF25F00E0EF76E240EF66E00EEEE
:1043800041F0A9EC02F0D8A4CAEF21F054EC3FF0C0
:1043900017EF25F00E0EF76E280EF66E00EE41F0C8
:1043A000A9EC02F0D8A4D9EF21F09AEC3FF017EF76
:1043B00025F00E0EF76E2C0EF66E00EE41F0A9EC15
:1043C00002F0D8A4E8EF21F027EC2AF017EF25F04F
:1043D0000E0EF76E300EF66E00EE41F0A9EC02F014
:1043E000D8A4F7EF21F036EC2AF017EF25F00E0EE7
:1043F000F76E360EF66E00EE41F0A9EC02F0D8A48E
:1044000006EF22F060EC2AF017EF25F00E0EF76EA3
:104410003A0EF66E00EE41F0A9EC02F0D8A415EFCA
:1044200022F048EC36F017EF25F00E0EF76E3E0E38
:10443000F66E00EE41F0A9EC02F0D8A424EF22F0D1
:10444000F4EC36F017EF25F00E0EF76E460EF66E12
:1044500000EE41F0A9EC02F0D8A433EF22F0C3EC57
:1044600030F017EF25F00E0EF76E4E0EF66E00EEE2
:1044700041F0A9EC02F0D8A442EF22F0FEEC30F0BB
:1044800017EF25F00E0EF76E560EF66E00EE41F0A9
:10449000A9EC02F0D8A451EF22F039EC31F017EF7B
:1044A00025F00E0EF76E5E0EF66E00EE41F0A9ECF2
:1044B00002F0D8A460EF22F074EC31F017EF25F091
:1044C0000E0EF76E660EF66E00EE41F0A9EC02F0ED
:1044D000D8A46FEF22F0AFEC31F017EF25F00E0EFD
:1044E000F76E6E0EF66E00EE41F0A9EC02F0D8A465
:1044F0007EEF22F0EAEC31F017EF25F00E0EF76EAA
:10450000760EF66E00EE41F0A9EC02F0D8A48DEF25
:1045100022F025EC32F017EF25F00E0EF76E7E0E2E
:10452000F66E00EE41F0A9EC02F0D8A49CEF22F068
:1045300060EC32F017EF25F00E0EF76E860EF66E79
:1045400000EE41F0A9EC02F0D8A4ABEF22F08EEC23
:1045500030F017EF25F00E0EF76E8E0EF66E00EEB1
:1045600041F0A9EC02F0D8A4BAEF22F09BEC32F0B3
:1045700017EF25F00E0EF76E960EF66E00EE41F078
:10458000A9EC02F0D8A4C9EF22F0F0EC32F017EF5A
:1045900025F00E0EF76E9E0EF66E00EE41F0A9ECC1
:1045A00002F0D8A4D8EF22F045EC33F017EF25F055
:1045B0000E0EF76EA60EF66E00EE41F0A9EC02F0BC
:1045C000D8A4E7EF22F09AEC33F017EF25F00E0EA7
:1045D000F76EAE0EF66E00EE41F0A9EC02F0D8A434
:1045E000F6EF22F091EC3BF017EF25F00E0EF76E90
:1045F000B60EF66E00EE41F0A9EC02F0D8A405EF7D
:1046000023F0AFEC3BF017EF25F00E0EF76EC00E67
:10461000F66E00EE41F0A9EC02F0D8A414EF23F0FE
:10462000CBEC29F017EF25F00E0EF76EC40EF66EE8
:1046300000EE41F0A9EC02F0D8A423EF23F0C3EC84
:1046400029F017EF25F00E0EF76ECA0EF66E00EE8B
:1046500041F0A9EC02F0D8A432EF23F0E8EC4CF0E2
:1046600017EF25F00E0EF76ED00EF66E00EE41F04D
:10467000A9EC02F0D8A441EF23F0D4EC43F017EFFB
:1046800025F00E0EF76ED60EF66E00EE41F0A9EC98
:1046900002F0D8A450EF23F0C1EC40F017EF25F062
:1046A0000E0EF76EDC0EF66E00EE41F0A9EC02F095
:1046B000D8A45FEF23F08CEC47F017EF25F00E0E37
:1046C000F76EE40EF66E00EE41F0A9EC02F0D8A40D
:1046D0006EEF23F0D6EC25F017EF25F00E0EF76EF7
:1046E000EA0EF66E00EE41F0A9EC02F0D8A489EFD4
:1046F00023F00101D78104EEA2F00E0EF76EF20E48
:10470000F66E81EC02F0EF6A000165EC1DF017EF28
:1047100025F00F0EF76E000EF66E00EE41F0A9ECDC
:1047200002F0D8A4A4EF23F00101D79104EEA2F087
:104730000F0EF76E0A0EF66E81EC02F0EF6A0001C2
:1047400065EC1DF017EF25F00F0EF76E1A0EF66EE2
:1047500000EE41F0A9EC02F0D8A4BFEF23F0010174
:10476000D78304EEA2F00F0EF76E240EF66E81ECE6
:1047700002F0EF6A000165EC1DF017EF25F00F0E57
:10478000F76E420EF66E00EE41F0A9EC02F0D8A4EE
:10479000DAEF23F00101D79304EEA2F00F0EF76ECB
:1047A0004E0EF66E81EC02F0EF6A000165EC1DF032
:1047B00017EF25F00F0EF76E6C0EF66E00EE41F05F
:1047C000A9EC02F0D8A4F5EF23F00101D78504EE9F
:1047D000A2F00F0EF76E780EF66E81EC02F0EF6A23
:1047E000000165EC1DF017EF25F00F0EF76E8E0E31
:1047F000F66E00EE41F0A9EC02F0D8A410EF24F020
:104800000101D79504EEA2F00F0EF76E9A0EF66E28
:1048100081EC02F0EF6A000165EC1DF017EF25F066
:104820000F0EF76EB20EF66E00EE41F0A9EC02F03C
:10483000D8A41FEF24F01EEC25F017EF25F00F0E83
:10484000F76EB80EF66E00EE41F0A9EC02F0D8A4B7
:104850002EEF24F051EC25F017EF25F00F0EF76E38
:10486000C20EF66E00EE41F0A9EC02F0D8A43DEFC6
:1048700024F049EC29F017EF25F00F0EF76ECC0E5F
:10488000F66E00EE41F0A9EC02F0D8A44CEF24F053
:10489000D3EC29F017EF25F00F0EF76ED60EF66E5B
:1048A00000EE41F0A9EC02F0D8A45BEF24F0D3ECC9
:1048B00029F017EF25F00F0EF76EDA0EF66E00EE08
:1048C00041F0A9EC02F0D8A476EF24F00401A16B2A
:1048D00004EEA2F00F0EF76EE40EF66E81EC02F01D
:1048E000EF6A000165EC1DF017EF25F0100EF76E72
:1048F000000EF66E00EE41F0A9EC02F0D8A492EFA3
:1049000024F0010E0401A16F04EEA2F0100EF76E68
:10491000080EF66E81EC02F0EF6A000165EC1DF006
:1049200017EF25F0100EF76E320EF66E00EE41F026
:10493000A9EC02F0D8A4A1EF24F0BBEC1BF017EF18
:1049400025F0100EF76E380EF66E00EE41F0A9EC71
:1049500002F0D8A4B0EF24F026EC40F017EF25F0D9
:10496000100EF76E3E0EF66E00EE41F0A9EC02F06E
:10497000D8A4BFEF24F0EBEF14F017EF25F0100EE2
:10498000F76E460EF66E00EE41F0A9EC02F0D8A4E8
:10499000CEEF24F0CDEC3BF017EF25F0100EF76EC4
:1049A0004E0EF66E00EE41F0A9EC02F0D8A4DDEF59
:1049B00024F0E2EC3BF017EF25F0100EF76E560EE8
:1049C000F66E00EE41F0A9EC02F0D8A4ECEF24F072
:1049D000CCEC2FF017EF25F0100EF76E5A0EF66E96
:1049E00000EE41F0A9EC02F0D8A4FBEF24F01AECA1
:1049F0003BF017EF25F0100EF76E620EF66E00EE2C
:104A000041F0A9EC02F0D8A40AEF25F03EEC3BF00F
:104A100017EF25F0100EF76E680EF66E00EE41F0FF
:104A2000A9EC02F0D8A417EF25F0F1EC3AF004015C
:104A3000A06B9F6B000184EC17F0120002EEC8F02F
:104A4000100EF76E6E0EF66E81EC02F011EEDAF0DB
:104A5000040EE75204E0E6CFEEFFE82EFAD7100E80
:104A6000F76E760EF66E81EC02F015EEDAF0060EB9
:104A7000E75204E0E6CFEEFFE82EFAD7100EF76E0D
:104A8000800EF66E81EC02F0020E016E0501E3511C
:104A9000CCEC00F0EF6A0001CCEC1BF05AEC1EF0FD
:104AA00012000501E3510A0DF3CF1AF0F4CF1BF009
:104AB000CEEC01F00001C2DF12000401A15300019D
:104AC000D8A497EF25F002EEC8F0100EF76E8C0E0A
:104AD000F66E81EC02F0020E016EE86A82B8010EF9
:104AE000CCEC00F0020E016EE86A82BA010ECCEC4A
:104AF00000F0020E016EE86A81B0010ECCEC00F00D
:104B0000020E016EE86A81B2010ECCEC00F0020EDA
:104B1000016EE86A81B4010ECCEC00F0300EEE6E4E
:104B2000EE6EEE6EEF6ACCEC1BF05AEC1EF0010E4E
:104B30000401A15D0001D8A4D2EF25F002EEC8F077
:104B4000100EF76E940EF66E81EC02F0020E016EFE
:104B5000E86A82B8010ECCEC00F0020E016EE86A41
:104B600082BA010ECCEC00F0020E016EE86A81B050
:104B7000010ECCEC00F0020E016EE86A81B2010E6B
:104B8000CCEC00F0020E016EE86A81B4010ECCECB0
:104B900000F0300EEE6EEE6EEE6EEF6ACCEC1BF0B7
:104BA0005AEC1EF0140ECCEC01F012000401A153DB
:104BB0000001D8A464EF27F002EEC8F0100EF76EE3
:104BC0009C0EF66E81EC02F0020E016EE86A82B86D
:104BD000010ECCEC00F0020E016EE86A82BA010E02
:104BE000CCEC00F0020E016EE86A81B0010ECCEC54
:104BF00000F0020E016EE86A81B2010ECCEC00F00A
:104C0000020E016EE86A81B4010ECCEC00F0300EA9
:104C1000EE6EEE6EEE6EEF6ACCEC1BF05AEC1EF010
:104C2000140ECCEC01F002EEC8F0100EF76EA40EDC
:104C3000F66E81EC02F0020E016E38C52DF037C51C
:104C40002CF036C52BF035C52AF0030EFEEC00F033
:104C50002C0EEE6E020E016E3CC52DF03BC52CF005
:104C60003AC52BF039C52AF0030EFEEC00F02C0EED
:104C7000EE6E020E016E40C52DF03FC52CF03EC514
:104C80002BF03DC52AF0030EFEEC00F02C0EEE6E6C
:104C9000020E016E44C52DF043C52CF042C52BF029
:104CA00041C52AF0030EFEEC00F0EF6ACCEC1BF0DD
:104CB0005AEC1EF0140ECCEC01F002EEC8F0100E0F
:104CC000F76EAC0EF66E81EC02F0020E016E066A13
:104CD000EAC51FF0E9C51EF0CFEC00F02C0EEE6E19
:104CE000020E016E066AECC51FF0EBC51EF0CFEC9C
:104CF00000F02C0EEE6E020E016E066AEEC51FF07D
:104D0000EDC51EF0CFEC00F02C0EEE6E020E016E23
:104D1000066AF0C51FF0EFC51EF0CFEC00F02C0EB8
:104D2000EE6E020E016E066AF2C51FF0F1C51EF0AE
:104D3000CFEC00F02C0EEE6E020E016E066AF4C58A
:104D40001FF0F3C51EF0CFEC00F02C0EEE6E020E3D
:104D5000016E066AF6C51FF0F5C51EF0CFEC00F037
:104D60002C0EEE6E020E016E000ECCEC00F02C0E3E
:104D7000EE6E020E016EE86A060105B9010ECCEC7A
:104D800000F0EF6A0001CCEC1BF05AEC1EF0140EA0
:104D9000CCEC01F002EEC8F0100EF76EB40EF66E19
:104DA00081EC02F0020E016E066AF8C51FF0F7C52D
:104DB0001EF0CFEC00F02C0EEE6E020E016E066AB5
:104DC000FAC51FF0F9C51EF0CFEC00F02C0EEE6E08
:104DD000020E016E066AFCC51FF0FBC51EF0CFEC8B
:104DE00000F02C0EEE6E020E016E066AFEC51FF07C
:104DF000FDC51EF0CFEC00F02C0EEE6E020E016E23
:104E0000066A00C61FF0FFC51EF0CFEC00F02C0EA6
:104E1000EE6E020E016E066A02C61FF001C61EF09B
:104E2000CFEC00F02C0EEE6E020E016E066A04C688
:104E30001FF003C61EF0CFEC00F02C0EEE6E020E3B
:104E4000016E000ECCEC00F02C0EEE6E020E016E28
:104E5000E86A060105BB010ECCEC00F0EF6A000128
:104E6000CCEC1BF05AEC1EF0140ECCEC01F002EE70
:104E7000C8F0100EF76EBC0EF66E81EC02F0020E5A
:104E8000016E0501E351CCEC00F02C0EEE6E020E2B
:104E9000016E066AD7C51FF0D6C51EF0CFEC00F034
:104EA0002C0EEE6E020E016E066AD9C51FF0D8C533
:104EB0001EF0CFEC00F0EF6A0001CCEC1BF05AECD6
:104EC0001EF0140ECCEC01F0010E0401A15D0001F6
:104ED000D8A4F3EF28F002EEC8F0100EF76EC40E5F
:104EE000F66E81EC02F0020E016EE86A82B8010EE5
:104EF000CCEC00F0020E016EE86A82BA010ECCEC36
:104F000000F0020E016EE86A81B0010ECCEC00F0F8
:104F1000020E016EE86A81B2010ECCEC00F0020EC6
:104F2000016EE86A81B4010ECCEC00F0300EEE6E3A
:104F3000EE6EEE6EEF6ACCEC1BF05AEC1EF0140E27
:104F4000CCEC01F002EEC8F0100EF76ECC0EF66E4F
:104F500081EC02F0020E016E38C52DF037C52CF041
:104F600036C52BF035C52AF0030EFEEC00F02C0EF2
:104F7000EE6E020E016E3CC52DF03BC52CF03AC51D
:104F80002BF039C52AF0030EFEEC00F02C0EEE6E6D
:104F9000020E016E40C52DF03FC52CF03EC52BF032
:104FA0003DC52AF0030EFEEC00F02C0EEE6E020E54
:104FB000016E44C52DF043C52CF042C52BF041C510
:104FC0002AF0030EFEEC00F0EF6ACCEC1BF05AEC7A
:104FD0001EF0140ECCEC01F002EEC8F0100EF76ECD
:104FE000D40EF66E81EC02F0020E016E066AEAC57E
:104FF0001FF0E9C51EF0CFEC00F02C0EEE6E020E95
:10500000016E066AECC51FF0EBC51EF0CFEC00F098
:105010002C0EEE6E020E016E066AEEC51FF0EDC597
:105020001EF0CFEC00F02C0EEE6E020E016E066A42
:10503000F0C51FF0EFC51EF0CFEC00F02C0EEE6EA9
:10504000020E016E066AF2C51FF0F1C51EF0CFEC2C
:1050500000F02C0EEE6E020E016E066AF4C51FF013
:10506000F3C51EF0CFEC00F02C0EEE6E020E016EBA
:10507000066AF6C51FF0F5C51EF0CFEC00F02C0E49
:10508000EE6E020E016E000ECCEC00F02C0EEE6EF9
:10509000020E016EE86A060105B9010ECCEC00F0C3
:1050A000EF6A0001CCEC1BF05AEC1EF0140ECCECB5
:1050B00001F002EEC8F0100EF76EDC0EF66E81EC19
:1050C00002F0020E016E066AF8C51FF0F7C51EF069
:1050D000CFEC00F02C0EEE6E020E016E066AFAC5E1
:1050E0001FF0F9C51EF0CFEC00F02C0EEE6E020E94
:1050F000016E066AFCC51FF0FBC51EF0CFEC00F088
:105100002C0EEE6E020E016E066AFEC51FF0FDC586
:105110001EF0CFEC00F02C0EEE6E020E016E066A51
:1051200000C61FF0FFC51EF0CFEC00F02C0EEE6E97
:10513000020E016E066A02C61FF001C61EF0CFEC19
:1051400000F02C0EEE6E020E016E066A04C61FF011
:1051500003C61EF0CFEC00F02C0EEE6E020E016EB8
:10516000000ECCEC00F02C0EEE6E020E016EE86A22
:10517000060105BB010ECCEC00F0EF6A0001CCEC9F
:105180001BF05AEC1EF0140ECCEC01F002EEC8F04D
:10519000100EF76EE40EF66E81EC02F0020E016E58
:1051A0000501E351CCEC00F02C0EEE6E020E016E08
:1051B000066AD7C51FF0D6C51EF0CFEC00F02C0E46
:1051C000EE6E020E016E066AD9C51FF0D8C51EF03C
:1051D000CFEC00F0EF6A0001CCEC1BF05AEC1EF0B3
:1051E000140ECCEC01F01200100EF76EEC0EF66E01
:1051F00001EEDAF0A9EC02F0D8A41BEF29F0010EC1
:105200000101CA6F0001040E0101CA5D0001D8B09E
:1052100019EF29F094928292FA0ECCEC01F094925C
:105220008282FA0ECCEC01F00101CA2B0001D8A455
:10523000E9D748EF29F0010E0101CA6F0001030E02
:105240000101CA5D0001D8B048EF29F09492829222
:10525000010E1B6EF40ECDEC01F094928282C80E0A
:10526000CCEC01F094928292010E1B6EF40ECDEC08
:1052700001F094928282C80ECCEC01F0010E1B6EFC
:10528000900ECDEC01F00101CA2B0001D8A4D6D7B5
:10529000120001EEDAF0460EEE6E410EEE6E490E91
:1052A000EE6E4C0EEE6EEF6A1200BCEC29F001EED1
:1052B0002FF0100EF76EF00EF66E81EC02F0020E7B
:1052C000016E0501E351CCEC00F0110EF76E040EF7
:1052D000F66E81EC02F0EF6A0001BBEC1BF0010EF0
:1052E0000101CA6F0001040E0101CA5D0001D8B0BE
:1052F0009FEF29F094928292820E026E040E076E46
:10530000010E046EF40E036E030E1F6EE80E1E6E89
:1053100033EC00F094928282820E026E040E076ECD
:10532000010E046EF40E036E010E1F6E900E1E6EC3
:1053300033EC00F00101CA2B0001D8A4D3D705EE4D
:1053400090F0460EEE6E410EEE6E490EEE6E4C0E75
:10535000EE6EEF6A82EC2AF094928292010E1B6E3E
:10536000F40ECDEC01F094928282010E1B6EF40ECD
:10537000CDEC01F0F1D712008298829A819081924F
:105380008194120012000501236B0101696B060173
:10539000059700011200010E0501236F010E0101A6
:1053A000696F00011200E8DF2D0E0101CA6F010EC6
:1053B000D26F0001090E0101D25D0001D8B025EFC6
:1053C0002AF0949882880101CA51CCEC01F094989B
:1053D0008298949A828ACA51CCEC01F0949A829A6B
:1053E00093908180CA51CCEC01F09390819093927C
:1053F0008182CA51CCEC01F0939281929394818482
:10540000CA51CCEC01F09394819493928182CA5159
:10541000CCEC01F09392819293908180CA51CCECB4
:1054200001F093908190949A828ACA51CCEC01F059
:10543000949A829A94988288CA51CCEC01F09498FC
:105440008298D22B0001D8A4B4D796DF120005EEC3
:1054500090F011EE2FF0360EE75204E0E6CFEEFFAB
:10546000E82EFAD7EF6A82EC2AF01200110EF76EDE
:10547000160EF66E01EE2FF0A9EC02F0D8A451EF53
:105480002AF00501288504EEA2F0110EF76E1A0E1F
:10549000F66E81EC02F0EF6A000165EC1DF05FEF43
:1054A0002AF00501289504EEA2F0110EF76E280EE1
:1054B000F66E81EC02F0EF6A000165EC1DF012005F
:1054C00001EE2FF084EC00F005018E6F040E176ED4
:1054D000B00E166E1B6A8EC51AF044EC02F08C6F8B
:1054E00017C08DF504EEA2F0110EF76E380EF66EB1
:1054F00081EC02F0020E016E8E51CCEC00F0EF6AEE
:105500000001120004EEA2F0110EF76E4A0EF66EC4
:1055100081EC02F015EE90F0320EE75204E0E6CF97
:10552000EEFFE82EFAD7EF6A65EC1DF0040E176E59
:10553000B00E166E1B6A8EC51AF044EC02F005011F
:105540008C6F17C08DF59492828205EE90F0E86A18
:10555000EE5202E0E83EFCD78F6F010E0101CA6FE8
:1055600000010101CA5105018F5D0001D8A07CEF47
:105570002DF005EEC3F015EE90F0CAC1F3FF010E59
:1055800089EC02F0EF6A410E0501C35D0001D8A469
:10559000D3EF2AF005EEC8F02E0EEE6E2D0EEE6E55
:1055A000EF6A74EF2DF0420E0501C35D0001D8A42F
:1055B000E5EF2AF005EEC8F02D0EEE6E2E0EEE6E23
:1055C000EE6EEE6EEF6A74EF2DF0430E0501C35DD3
:1055D0000001D8A4F9EF2AF005EEC8F02D0EEE6E0A
:1055E0002E0EEE6E2D0EEE6E2E0EEE6EEF6A74EF38
:1055F0002DF0440E0501C35D0001D8A40AEF2BF085
:1056000005EEC8F02D0EEE6E2E0EEE6EEE6EEF6A0B
:1056100074EF2DF0450E0501C35D0001D8A418EF0D
:105620002BF005EEC8F02E0EEE6EEF6A74EF2DF043
:10563000460E0501C35D0001D8A42BEF2BF005EE4B
:10564000C8F02E0EEE6EEE6E2D0EEE6E2E0EEE6E7F
:10565000EF6A74EF2DF0470E0501C35D0001D8A479
:105660003CEF2BF005EEC8F02D0EEE6EEE6E2E0E1A
:10567000EE6EEF6A74EF2DF0480E0501C35D000178
:10568000D8A44DEF2BF005EEC8F02E0EEE6EEE6EA8
:10569000EE6EEE6EEF6A74EF2DF0490E0501C35DFC
:1056A0000001D8A45CEF2BF005EEC8F02E0EEE6ED4
:1056B000EE6EEF6A74EF2DF04A0E0501C35D000136
:1056C000D8A46EEF2BF005EEC8F02E0EEE6E2D0E68
:1056D000EE6EEE6EEE6EEF6A74EF2DF04B0E05017E
:1056E000C35D0001D8A480EF2BF005EEC8F02D0EAD
:1056F000EE6E2E0EEE6E2D0EEE6EEF6A74EF2DF046
:105700004C0E0501C35D0001D8A493EF2BF005EE0C
:10571000C8F02E0EEE6E2D0EEE6E2E0EEE6EEE6EAE
:10572000EF6A74EF2DF04D0E0501C35D0001D8A4A2
:10573000A2EF2BF005EEC8F02D0EEE6EEE6EEF6AC6
:1057400074EF2DF04E0E0501C35D0001D8A4B2EF39
:105750002BF005EEC8F02D0EEE6E2E0EEE6EEF6AFB
:1057600074EF2DF04F0E0501C35D0001D8A4C2EF08
:105770002BF005EEC8F02D0EEE6EEE6EEE6EEF6ABB
:1057800074EF2DF0500E0501C35D0001D8A4D5EFD4
:105790002BF005EEC8F02E0EEE6E2D0EEE6EEE6EB8
:1057A0002E0EEE6EEF6A74EF2DF0510E0501C35D03
:1057B0000001D8A4E8EF2BF005EEC8F02D0EEE6E38
:1057C000EE6E2E0EEE6E2D0EEE6EEF6A74EF2DF075
:1057D000520E0501C35D0001D8A4FAEF2BF005EECF
:1057E000C8F02E0EEE6E2D0EEE6E2E0EEE6EEF6AE1
:1057F00074EF2DF0530E0501C35D0001D8A40AEF2C
:105800002CF005EEC8F02E0EEE6EEE6EEE6EEF6A28
:1058100074EF2DF0540E0501C35D0001D8A418EFFC
:105820002CF005EEC8F02D0EEE6EEF6A74EF2DF041
:10583000550E0501C35D0001D8A429EF2CF005EE3B
:10584000C8F02E0EEE6EEE6E2D0EEE6EEF6A74EF59
:105850002DF0560E0501C35D0001D8A43BEF2CF0DE
:1058600005EEC8F02E0EEE6EEE6EEE6E2D0EEE6EA6
:10587000EF6A74EF2DF0570E0501C35D0001D8A447
:105880004CEF2CF005EEC8F02E0EEE6E2D0EEE6EE7
:10589000EE6EEF6A74EF2DF0580E0501C35D000146
:1058A000D8A45FEF2CF005EEC8F02D0EEE6E2E0E94
:1058B000EE6EEE6E2D0EEE6EEF6A74EF2DF0590E59
:1058C0000501C35D0001D8A472EF2CF005EEC8F00D
:1058D0002D0EEE6E2E0EEE6E2D0EEE6EEE6EEF6A4D
:1058E00074EF2DF05A0E0501C35D0001D8A484EFBA
:1058F0002CF005EEC8F02D0EEE6EEE6E2E0EEE6E56
:10590000EE6EEF6A74EF2DF0300E0501C35D0001FD
:10591000D8A496EF2CF005EEC8F02D0EEE6EEE6ECC
:10592000EE6EEE6EEE6EEF6A74EF2DF0310E050145
:10593000C35D0001D8A4A9EF2CF005EEC8F02E0E2F
:10594000EE6E2D0EEE6EEE6EEE6EEE6EEF6A74EF94
:105950002DF0320E0501C35D0001D8A4BCEF2CF080
:1059600005EEC8F02E0EEE6EEE6E2D0EEE6EEE6EA5
:10597000EE6EEF6A74EF2DF0330E0501C35D00018A
:10598000D8A4CFEF2CF005EEC8F02E0EEE6EEE6E22
:10599000EE6E2D0EEE6EEE6EEF6A74EF2DF0340E9D
:1059A0000501C35D0001D8A4E1EF2CF005EEC8F0BD
:1059B0002E0EEE6EEE6EEE6E2D0EEE6EEF6A74EF44
:1059C0002DF0350E0501C35D0001D8A4F3EF2CF0D6
:1059D00005EEC8F02E0EEE6EEE6EEE6EEE6EEE6E14
:1059E000EF6A74EF2DF0360E0501C35D0001D8A4F7
:1059F00006EF2DF005EEC8F02D0EEE6E2E0EEE6EBB
:105A0000EE6EEE6EEE6EEF6A74EF2DF0370E05015E
:105A1000C35D0001D8A419EF2DF005EEC8F02D0EDE
:105A2000EE6EEE6E2E0EEE6EEE6EEE6EEF6A74EFB2
:105A30002DF0380E0501C35D0001D8A42CEF2DF028
:105A400005EEC8F02D0EEE6EEE6EEE6E2E0EEE6EC4
:105A5000EE6EEF6A74EF2DF0390E0501C35D0001A3
:105A6000D8A43FEF2DF005EEC8F02D0EEE6EEE6ED1
:105A7000EE6EEE6E2E0EEE6EEF6A74EF2DF02F0EC0
:105A80000501C35D0001D8A454EF2DF005EEC8F068
:105A90002D0EEE6E2E0EEE6EEE6E2D0EEE6E2E0EA8
:105AA000EE6EEF6A74EF2DF03D0E0501C35D00014F
:105AB000D8A468EF2DF005EEC8F02D0EEE6E2E0E78
:105AC000EE6EEE6EEE6E2D0EEE6EEF6A74EF2DF052
:105AD000200E0501C35D0001D8A474EF2DF005EE82
:105AE000C8F0200EEE6EEF6A7DEC2DF00101CA2B9E
:105AF0000001D8A4B0EF2AF0120005EEC8F0E86A61
:105B0000EE5202E0E83EFCD70101D26F010ED56FE4
:105B100000010101D551D25D0001D8A01EEF2EF089
:105B200005EEC5F015EEC8F0D5C1F3FF010E89EC06
:105B300002F0EF6A2E0E0501C55D0001D8A4C9EF81
:105B40002DF094928292D896050128A5D88600015E
:105B5000D8B6ADEF2DF093948184820E026E040EC0
:105B6000076E8DC504F08CC503F08BC51FF08AC588
:105B70001EF033EC00F0D896050128A5D886000168
:105B8000D8B6C5EF2DF0939481949492828213EF4E
:105B90002EF02D0E0501C55D0001D8A4FEEF2DF0FD
:105BA00094928292D896050128A5D8860001D8B68D
:105BB000DCEF2DF093948184820E026E040E076E4A
:105BC00005018D51030DF3CF04F08C51030DF3CF7C
:105BD00003F0F45004268BC51FF08AC51EF033EC89
:105BE00000F0D89628A5D8860001D8B6FAEF2DF097
:105BF000939481949492828213EF2EF0200E0501EB
:105C0000C55D0001D8A412EF2EF005018D51030DE2
:105C1000F3CF1BF08C51030DF3CF1AF0F4501B2679
:105C2000CEEC01F000018DC51BF005018C51CDECCF
:105C300001F00101D52B0001D8A46AD705018D51CF
:105C4000030DF3CF1BF08C51030DF3CF1AF0F4507A
:105C50001B26CEEC01F000011200000EB5EC01F0A5
:105C600005012D6F2BC02EF5156A146A136A8F0E6D
:105C7000126E2EC50FF02DC50EF078EC04F0C0ECBE
:105C800003F011C0D0F110C0CFF10FC0CEF10EC0A3
:105C9000CDF1116A106A200E0F6E810E0E6ED0C10A
:105CA00015F0CFC114F0CEC113F0CDC112F028EC25
:105CB00004F011C02DF010C02CF00FC02BF00EC05E
:105CC0002AF02DC011F02CC010F02BC00FF02AC00C
:105CD0000EF02CC515F02BC514F02AC513F029C5FC
:105CE00012F028EC04F011C038F510C037F50FC0E1
:105CF00036F50EC035F538C511F037C510F036C58C
:105D00000FF035C50EF048C515F047C514F046C56F
:105D100013F045C512F026EC03F011C038F510C0A1
:105D200037F50FC036F50EC035F5010EB5EC01F0B4
:105D30002F6F2BC030F5156A146A136A8F0E126E1E
:105D400030C50FF02FC50EF078EC04F0C0EC03F076
:105D500011C0D0F110C0CFF10FC0CEF10EC0CDF107
:105D6000116A106A200E0F6E810E0E6ED0C115F0F2
:105D7000CFC114F0CEC113F0CDC112F028EC04F065
:105D800011C02DF010C02CF00FC02BF00EC02AF067
:105D90002DC011F02CC010F02BC00FF02AC00EF057
:105DA0002CC515F02BC514F02AC513F029C512F027
:105DB00028EC04F011C03CF510C03BF50FC03AF5DB
:105DC0000EC039F53CC511F03BC510F03AC50FF0D7
:105DD00039C50EF04CC515F04BC514F04AC513F08B
:105DE00049C512F026EC03F011C03CF510C03BF59C
:105DF0000FC03AF50EC039F5020EB5EC01F0316F67
:105E00002BC032F5156A146A136A8F0E126E32C5F2
:105E10000FF031C50EF078EC04F0C0EC03F011C0C7
:105E2000D0F110C0CFF10FC0CEF10EC0CDF1116A8C
:105E3000106A200E0F6E810E0E6ED0C115F0CFC10C
:105E400014F0CEC113F0CDC112F028EC04F011C053
:105E50002DF010C02CF00FC02BF00EC02AF02DC07A
:105E600011F02CC010F02BC00FF02AC00EF02CC582
:105E700015F02BC514F02AC513F029C512F028EC33
:105E800004F011C040F510C03FF50FC03EF50EC044
:105E90003DF540C511F03FC510F03EC50FF03DC5C2
:105EA0000EF050C515F04FC514F04EC513F04DC59A
:105EB00012F026EC03F011C040F510C03FF50FC002
:105EC0003EF50EC03DF5030EB5EC01F0336F2BC06F
:105ED00034F5156A146A136A8F0E126E34C50FF00A
:105EE00033C50EF078EC04F0C0EC03F011C0D0F133
:105EF00010C0CFF10FC0CEF10EC0CDF1116A106A03
:105F0000200E0F6E810E0E6ED0C115F0CFC114F0B1
:105F1000CEC113F0CDC112F028EC04F011C02DF069
:105F200010C02CF00FC02BF00EC02AF02DC011F0C5
:105F30002CC010F02BC00FF02AC00EF02CC515F0AD
:105F40002BC514F02AC513F029C512F028EC04F073
:105F500011C044F510C043F50FC042F50EC041F525
:105F600044C511F043C510F042C50FF041C50EF015
:105F700054C515F053C514F052C513F051C512F0B5
:105F800026EC03F011C044F510C043F50FC042F5F4
:105F90000EC041F50001120004EEA2F0110EF76EE2
:105FA000540EF66E81EC02F0EF6A65EC1DF00A0EFD
:105FB000CCEC01F052DE04EEA2F0110EF76E7A0E78
:105FC000F66E81EC02F0020E016E38C52DF037C579
:105FD0002CF036C52BF035C52AF0030EFEEC00F090
:105FE000110EF76E8A0EF66E81EC02F0020E016E53
:105FF000066A2EC51FF02DC51EF0CFEC00F0290E4D
:10600000EE6EEF6A65EC1DF004EEA2F0110EF76E75
:10601000940EF66E81EC02F0020E016E3CC52DF07E
:106020003BC52CF03AC52BF039C52AF0030EFEEC27
:1060300000F0110EF76EA40EF66E81EC02F0020E67
:10604000016E066A30C51FF02FC51EF0CFEC00F0C0
:10605000290EEE6EEF6A65EC1DF004EEA2F0110E53
:10606000F76EAE0EF66E81EC02F0020E016E40C5C8
:106070002DF03FC52CF03EC52BF03DC52AF0030E98
:10608000FEEC00F0110EF76EBE0EF66E81EC02F023
:10609000020E016E066A32C51FF031C51EF0CFEC4C
:1060A00000F0290EEE6EEF6A65EC1DF004EEA2F032
:1060B000110EF76EC80EF66E81EC02F0020E016E44
:1060C00044C52DF043C52CF042C52BF041C52AF044
:1060D000030EFEEC00F0110EF76ED80EF66E81EC9A
:1060E00002F0020E016E066A34C51FF033C51EF0C1
:1060F000CFEC00F0290EEE6EEF6A65EC1DF004EEB9
:10610000A2F0110EF76EE20EF66E81EC02F0EF6A6D
:1061100065EC1DF00A0ECCEC01F01200120EF76EC9
:10612000080EF66E01EE2FF0A9EC02F0D8A4A8EF4D
:1061300030F0010E01016A6F04EEA2F0120EF76E4C
:106140000C0EF66E81EC02F0EF6A000165EC1DF0BA
:10615000120EF76E280EF66E01EE2FF0A9EC02F08B
:10616000D8A4C1EF30F001016A6B04EEA2F0120E68
:10617000F76E2C0EF66E81EC02F0EF6A000165EC12
:106180001DF01200120001EE2FF084EC00F01EC092
:106190000EF01FC00FF020C010F021C011F07AECFB
:1061A00004F011C058F510C057F50FC056F50EC0D9
:1061B00055F501EE9EF0020E016E58C52DF057C543
:1061C0002CF056C52BF055C52AF0030EFEEC00F05E
:1061D000EF6A04EEA2F0120EF76E480EF66E81EC36
:1061E00002F011EE9EF0140EE75204E0E6CFEEFF4F
:1061F000E82EFAD7EF6A65EC1DF0120001EE2FF0E1
:1062000084EC00F01EC00EF01FC00FF020C010F094
:1062100021C011F07AEC04F011C05CF510C05BF500
:106220000FC05AF50EC059F501EE9EF0020E016E38
:106230005CC52DF05BC52CF05AC52BF059C52AF072
:10624000030EFEEC00F0EF6A04EEA2F0120EF76E01
:106250005E0EF66E81EC02F011EE9EF0140EE75227
:1062600004E0E6CFEEFFE82EFAD7EF6A65EC1DF00A
:10627000120001EE2FF084EC00F01EC00EF01FC0E3
:106280000FF020C010F021C011F07AEC04F011C022
:1062900060F510C05FF50FC05EF50EC05DF501EE54
:1062A0009EF0020E016E60C52DF05FC52CF05EC53C
:1062B0002BF05DC52AF0030EFEEC00F0EF6A04EE51
:1062C000A2F0120EF76E740EF66E81EC02F011EE73
:1062D0009EF0140EE75204E0E6CFEEFFE82EFAD768
:1062E000EF6A65EC1DF0120001EE2FF084EC00F077
:1062F0001EC00EF01FC00FF020C010F021C011F022
:106300007AEC04F011C064F510C063F50FC062F5BB
:106310000EC061F501EE9EF0020E016E64C52DF017
:1063200063C52CF062C52BF061C52AF0030EFEECAC
:1063300000F0EF6A04EEA2F0120EF76E8A0EF66E0F
:1063400081EC02F011EE9EF0140EE75204E0E6CF6D
:10635000EEFFE82EFAD7EF6A65EC1DF0120001EEB1
:106360002FF084EC00F01EC00EF01FC00FF020C014
:1063700010F021C011F07AEC04F011C068F510C0E3
:1063800067F50FC066F50EC065F501EE9EF0020ED2
:10639000016E68C52DF067C52CF066C52BF065C58C
:1063A0002AF0030EFEEC00F0EF6A04EEA2F0120EEB
:1063B000F76EA00EF66E81EC02F011EE9EF0140E58
:1063C000E75204E0E6CFEEFFE82EFAD7EF6A65EC7D
:1063D0001DF0120001EE2FF084EC00F01EC00EF054
:1063E0001FC00FF020C010F021C011F07AEC04F0B3
:1063F00011C06CF510C06BF50FC06AF50EC069F5E1
:1064000001EE9EF0020E016E6CC52DF06BC52CF0F6
:106410006AC52BF069C52AF0030EFEEC00F0EF6AA6
:1064200004EEA2F0120EF76EB60EF66E81EC02F0DC
:1064300011EE9EF0140EE75204E0E6CFEEFFE82ED8
:10644000FAD7EF6A65EC1DF0120001EE2FF084EC34
:1064500000F01EC00EF01FC00FF020C010F021C0D1
:1064600011F07AEC04F011C070F510C06FF50FC098
:106470006EF50EC06DF501EE9EF0020E016E70C558
:106480002DF06FC52CF06EC52BF06DC52AF0030EF4
:10649000FEEC00F0EF6A04EEA2F0120EF76ECC0EE6
:1064A000F66E81EC02F011EE9EF0140EE75204E05D
:1064B000E6CFEEFFE82EFAD7EF6A65EC1DF012008A
:1064C00001EE2FF084EC00F01EC00EF01FC00FF0A4
:1064D00020C010F021C011F07AEC04F011C074F566
:1064E00010C073F50FC072F50EC071F501EE9EF08D
:1064F000020E016E74C52DF073C52CF072C52BF021
:1065000071C52AF0030EFEEC00F0EF6A04EEA2F073
:10651000120EF76EE20EF66E81EC02F011EE9EF0B6
:10652000140EE75204E0E6CFEEFFE82EFAD7EF6A4A
:1065300065EC1DF0120001EE2FF084EC00F01EC09F
:106540000EF01FC00FF020C010F021C011F07AEC47
:1065500004F011C0D0F110C0CFF10FC0CEF10EC0C9
:10656000CDF16F0E116E120E106E030E0F6E750EC2
:106570000E6ED0C115F0CFC114F0CEC113F0CDC155
:1065800012F028EC04F011C048F510C047F50FC018
:1065900046F50EC045F501EE9EF0020E016E48C5AF
:1065A0002DF047C52CF046C52BF045C52AF0030E4B
:1065B000FEEC00F0EF6A04EEA2F0120EF76EF80E99
:1065C000F66E81EC02F011EE9EF0140EE75204E03C
:1065D000E6CFEEFFE82EFAD7EF6A65EC1DF0120069
:1065E00001EE2FF084EC00F01EC00EF01FC00FF083
:1065F00020C010F021C011F07AEC04F011C0D0F1ED
:1066000010C0CFF10FC0CEF10EC0CDF16F0E116EE4
:10661000120E106E030E0F6E750E0E6ED0C115F0B9
:10662000CFC114F0CEC113F0CDC112F028EC04F0AC
:1066300011C04CF510C04BF50FC04AF50EC049F51E
:1066400001EE9EF0020E016E4CC52DF04BC52CF0F4
:106650004AC52BF049C52AF0030EFEEC00F0EF6AA4
:1066600004EEA2F0130EF76E1E0EF66E81EC02F031
:1066700011EE9EF0140EE75204E0E6CFEEFFE82E96
:10668000FAD7EF6A65EC1DF0120001EE2FF084ECF2
:1066900000F01EC00EF01FC00FF020C010F021C08F
:1066A00011F07AEC04F011C0D0F110C0CFF10FC09E
:1066B000CEF10EC0CDF16F0E116E120E106E030EE4
:1066C0000F6E750E0E6ED0C115F0CFC114F0CEC195
:1066D00013F0CDC112F028EC04F011C050F510C039
:1066E0004FF50FC04EF50EC04DF501EE9EF0020EB7
:1066F000016E50C52DF04FC52CF04EC52BF04DC589
:106700002AF0030EFEEC00F0EF6A04EEA2F0130E86
:10671000F76E440EF66E81EC02F011EE9EF0140E50
:10672000E75204E0E6CFEEFFE82EFAD7EF6A65EC19
:106730001DF0120001EE2FF084EC00F01EC00EF0F0
:106740001FC00FF020C010F021C011F07AEC04F04F
:1067500011C0D0F110C0CFF10FC0CEF10EC0CDF1FD
:106760006F0E116E120E106E030E0F6E750E0E6E02
:10677000D0C115F0CFC114F0CEC113F0CDC112F0CD
:1067800028EC04F011C054F510C053F50FC052F5B9
:106790000EC051F501EE9EF0020E016E54C52DF0B3
:1067A00053C52CF052C52BF051C52AF0030EFEEC58
:1067B00000F0EF6A04EEA2F0130EF76E6A0EF66EAA
:1067C00081EC02F011EE9EF0140EE75204E0E6CFE9
:1067D000EEFFE82EFAD7EF6A65EC1DF0120038C51F
:1067E00011F037C510F036C50FF035C50EF058C59D
:1067F00015F057C514F056C513F055C512F0B2EC9C
:1068000002F00108D8B41FEF34F0B0EC34F068C5E2
:1068100011F067C510F066C50FF065C50EF038C5FC
:1068200015F037C514F036C513F035C512F0B2ECCB
:1068300002F00108D8B41FEF34F07CEC35F03CC511
:1068400011F03BC510F03AC50FF039C50EF05CC52C
:1068500015F05BC514F05AC513F059C512F0B2EC2F
:1068600002F00108D8B44FEF34F0E3EC34F06CC51B
:1068700011F06BC510F06AC50FF069C50EF03CC58C
:1068800015F03BC514F03AC513F039C512F0B2EC5F
:1068900002F00108D8B44FEF34F0AFEC35F040C54A
:1068A00011F03FC510F03EC50FF03DC50EF060C5BC
:1068B00015F05FC514F05EC513F05DC512F0B2ECC3
:1068C00002F00108D8B47FEF34F016EC35F070C553
:1068D00011F06FC510F06EC50FF06DC50EF040C51C
:1068E00015F03FC514F03EC513F03DC512F0B2ECF3
:1068F00002F00108D8B47FEF34F0E2EC35F044C583
:1069000011F043C510F042C50FF041C50EF064C54B
:1069100015F063C514F062C513F061C512F0B2EC56
:1069200002F00108D8B4AFEF34F049EC35F074C58B
:1069300011F073C510F072C50FF071C50EF044C5AB
:1069400015F043C514F042C513F041C512F0B2EC86
:1069500002F00108D8B4AFEF34F015EC36F01200B5
:1069600004EEA2F0130EF76E900EF66E81EC02F0BC
:10697000020E016E58C52DF057C52CF056C52BF0F0
:1069800055C52AF0030EFEEC00F0130EF76EBC0E98
:10699000F66E81EC02F0020E016E38C52DF037C59F
:1069A0002CF036C52BF035C52AF0030EFEEC00F0B6
:1069B000760EEE6E2E0EEE6EEF6A65EC1DF0640E36
:1069C000CCEC01F0120004EEA2F0130EF76ECA0E2A
:1069D000F66E81EC02F0020E016E5CC52DF05BC517
:1069E0002CF05AC52BF059C52AF0030EFEEC00F02E
:1069F000130EF76EF60EF66E81EC02F0020E016ECB
:106A00003CC52DF03BC52CF03AC52BF039C52AF01A
:106A1000030EFEEC00F0760EEE6E2E0EEE6EEF6ABA
:106A200065EC1DF0640ECCEC01F0120004EEA2F057
:106A3000140EF76E040EF66E81EC02F0020E016E7B
:106A400060C52DF05FC52CF05EC52BF05DC52AF04A
:106A5000030EFEEC00F0140EF76E300EF66E81ECB5
:106A600002F0020E016E40C52DF03FC52CF03EC570
:106A70002BF03DC52AF0030EFEEC00F0760EEE6E14
:106A80002E0EEE6EEF6A65EC1DF0640ECCEC01F09C
:106A9000120004EEA2F0140EF76E3E0EF66E81ECBC
:106AA00002F0020E016E64C52DF063C52CF062C5C4
:106AB0002BF061C52AF0030EFEEC00F0140EF76E09
:106AC0006A0EF66E81EC02F0020E016E44C52DF0E6
:106AD00043C52CF042C52BF041C52AF0030EFEEC55
:106AE00000F0760EEE6E2E0EEE6EEF6A65EC1DF087
:106AF000640ECCEC01F0120004EEA2F0140EF76E5E
:106B0000780EF66E81EC02F0020E016E68C52DF073
:106B100067C52CF066C52BF065C52AF0030EFEECA8
:106B200000F0140EF76EA40EF66E81EC02F0020E69
:106B3000016E38C52DF037C52CF036C52BF035C5A4
:106B40002AF0030EFEEC00F0760EEE6E2E0EEE6EC8
:106B5000EF6A65EC1DF0640ECCEC01F0120004EE5F
:106B6000A2F0140EF76EB20EF66E81EC02F0020E79
:106B7000016E6CC52DF06BC52CF06AC52BF069C594
:106B80002AF0030EFEEC00F0140EF76EDE0EF66E29
:106B900081EC02F0020E016E3CC52DF03BC52CF0DD
:106BA0003AC52BF039C52AF0030EFEEC00F0760E44
:106BB000EE6E2E0EEE6EEF6A65EC1DF0640ECCEC00
:106BC00001F0120004EEA2F0140EF76EEC0EF66E59
:106BD00081EC02F0020E016E70C52DF06FC52CF035
:106BE0006EC52BF06DC52AF0030EFEEC00F0150EFD
:106BF000F76E180EF66E81EC02F0020E016E40C5C3
:106C00002DF03FC52CF03EC52BF03DC52AF0030EFC
:106C1000FEEC00F0760EEE6E2E0EEE6EEF6A65EC78
:106C20001DF0640ECCEC01F0120004EEA2F0150E83
:106C3000F76E260EF66E81EC02F0020E016E74C540
:106C40002DF073C52CF072C52BF071C52AF0030E20
:106C5000FEEC00F0150EF76E520EF66E81EC02F0AF
:106C6000020E016E44C52DF043C52CF042C52BF039
:106C700041C52AF0030EFEEC00F0760EEE6E2E0EED
:106C8000EE6EEF6A65EC1DF0640ECCEC01F01200C4
:106C9000150EF76E600EF66E01EE2FF0A9EC02F005
:106CA000D8A461EF36F00501756B04EEA2F0150E65
:106CB000F76E640EF66E81EC02F0EF6A000165EC8F
:106CC0001DF0150EF76E840EF66E01EE2FF0A9EC96
:106CD00002F0D8A47BEF36F0010E0501756F04EECB
:106CE000A2F0150EF76E880EF66E81EC02F0EF6AD8
:106CF000000165EC1DF0150EF76EAC0EF66E01EEA0
:106D00002FF0A9EC02F0D8A495EF36F0020E0501A1
:106D1000756F04EEA2F0150EF76EB40EF66E81ECF0
:106D200002F0EF6A000165EC1DF01200010E050192
:106D3000755D0001D8A4BBEF36F038C511F037C53A
:106D400010F036C50FF035C50EF03CC515F03BC54B
:106D500014F03AC513F039C512F0EAEC02F001085C
:106D6000D8B4B8EF36F0060105830001BAEF36F06B
:106D7000060105930001020E0501755D0001D8A40E
:106D8000F3EF36F03CC511F03BC510F03AC50FF0FB
:106D900039C50EF079C515F078C514F077C513F034
:106DA00076C512F0B2EC02F0336E3CC511F03BC573
:106DB00010F03AC50FF039C50EF038C515F037C5DB
:106DC00014F036C513F035C512F0B2EC02F03310F2
:106DD000D8B4F0EF36F0060105830001F2EF36F08B
:106DE000060105930001120001EE2FF084EC00F083
:106DF0001EC00EF01FC00FF020C010F021C011F017
:106E00007AEC04F011C079F510C078F50FC077F571
:106E10000EC076F5120012000101196B00019EAA46
:106E200014EF37F0AECF19F112009EB819EF37F01A
:106E3000FCD719C1ADFF120094928282D89601014D
:106E4000D7A1D8860001D8B632EF37F0150EF76E0D
:106E5000E40EF66E82EC01F00D0E8AEC01F00A0EE3
:106E60008AEC01F0D896060105ABD8860001D8B6A9
:106E700013EF38F081A83FEF37F0EDEF3AF0D896F6
:106E80000501E4A9D8860001D8B664EF37F0010106
:106E9000CC6B010ECB6F00010101CB510501FF5DF1
:106EA0000101CC51060100590001D8A062EF37F072
:106EB000010ECCEC01F00101CB2BD8B4CC2B00019E
:106EC000D8A4E9D79394819481A869EF37F0EDEFC6
:106ED0003AF0D8960501E4ABD8860001D8B68EEF1B
:106EE00037F00101CC6B010ECB6F00010101CB51DA
:106EF0000501FD5D0101CC510501FE590001D8A03D
:106F00008CEF37F0010ECCEC01F00101CB2BD8B4A3
:106F1000CC2B0001D8A4E9D79392819281A893EF5A
:106F200037F0EDEF3AF0D8960501E4ADD8860001D0
:106F3000D8B6B8EF37F00101CC6B010ECB6F000172
:106F40000101CB510501FB5D0101CC510501FC594B
:106F50000001D8A0B6EF37F0010ECCEC01F0010132
:106F6000CB2BD8B4CC2B0001D8A4E9D79390819037
:106F700081A8BDEF37F0EDEF3AF0D8960501E4AF08
:106F8000D8860001D8B6E2EF37F00101CC6B010ED4
:106F9000CB6F00010101CB510501F95D0101CC511D
:106FA0000501FA590001D8A0E0EF37F0010ECCEC52
:106FB00001F00101CB2BD8B4CC2B0001D8A4E9D728
:106FC000949A829A81A8E7EF37F0EDEF3AF0D896DD
:106FD000060105A1D8860001D8B60CEF38F00101F2
:106FE000CC6B010ECB6F00010101CB510501F75DA8
:106FF0000101CC510501F8590001D8A00AEF38F081
:10700000010ECCEC01F00101CB2BD8B4CC2B00014C
:10701000D8A4E9D79498829881A811EF38F0EDEFC1
:107020003AF0EAEF38F081A818EF38F0EDEF3AF0D7
:10703000D8960501E4A9D8860001D8B63DEF38F00E
:107040000101CC6B010ECB6F00010101CB51050199
:10705000F75D0101CC510501F8590001D8A03BEFC3
:1070600038F0010ECCEC01F00101CB2BD8B4CC2BC5
:107070000001D8A4E9D79498829881A842EF38F00B
:10708000EDEF3AF0D8960501E4ABD8860001D8B60A
:1070900067EF38F00101CC6B010ECB6F00010101ED
:1070A000CB510501F95D0101CC510501FA590001EF
:1070B000D8A065EF38F0010ECCEC01F00101CB2B2C
:1070C000D8B4CC2B0001D8A4E9D7949A829A81A88D
:1070D0006CEF38F0EDEF3AF0D8960501E4ADD886C4
:1070E0000001D8B691EF38F00101CC6B010ECB6FE7
:1070F00000010101CB510501FB5D0101CC510501EE
:10710000FC590001D8A08FEF38F0010ECCEC01F053
:107110000101CB2BD8B4CC2B0001D8A4E9D7939094
:10712000819081A896EF38F0EDEF3AF0D8960501FE
:10713000E4AFD8860001D8B6BBEF38F00101CC6BC4
:10714000010ECB6F00010101CB510501FD5D010175
:10715000CC510501FE590001D8A0B9EF38F0010E5D
:10716000CCEC01F00101CB2BD8B4CC2B0001D8A47E
:10717000E9D79392819281A8C0EF38F0EDEF3AF011
:10718000D896060105A1D8860001D8B6E5EF38F0FB
:107190000101CC6B010ECB6F00010101CB51050148
:1071A000FF5D0101CC51060100590001D8A0E3EFB9
:1071B00038F0010ECCEC01F00101CB2BD8B4CC2B74
:1071C0000001D8A4E9D79394819481A8EAEF38F01C
:1071D000EDEF3AF00501289DD896060105B7D8864F
:1071E0000001D8B6F6EF38F05DEC25F044EF17F06B
:1071F000D896060105A3D8860001D8B602EF39F06B
:1072000044EF17F094928282D8960101D7A1D886D4
:107210000001D8B618EF39F0150EF76EFC0EF66EB9
:1072200082EC01F00D0E8AEC01F00A0E8AEC01F0FE
:10723000D896060105A9D8860001D8B6F9EF39F02D
:1072400081A825EF39F0EDEF3AF0D8960501E4A9D1
:10725000D8860001D8B64AEF39F00101CC6B010E97
:10726000CB6F00010101CB510501E95D0101CC515A
:107270000501EA590001D8A048EF39F0010ECCEC25
:1072800001F00101CB2BD8B4CC2B0001D8A4E9D755
:107290009498828881A84FEF39F0EDEF3AF0D896B4
:1072A0000501E4ABD8860001D8B674EF39F00101CE
:1072B000CC6B010ECB6F00010101CB510501EB5DE1
:1072C0000101CC510501EC590001D8A072EF39F051
:1072D000010ECCEC01F00101CB2BD8B4CC2B00017A
:1072E000D8A4E9D7949A828A81A879EF39F0EDEF92
:1072F0003AF0D8960501E4ADD8860001D8B69EEFE5
:1073000039F00101CC6B010ECB6F00010101CB51B3
:107310000501ED5D0101CC510501EE590001D8A038
:107320009CEF39F0010ECCEC01F00101CB2BD8B46D
:10733000CC2B0001D8A4E9D79390818081A8A3EF3A
:1073400039F0EDEF3AF0D8960501E4AFD8860001A8
:10735000D8B6C8EF39F00101CC6B010ECB6F00013C
:107360000101CB510501EF5D0101CC510501F0593F
:107370000001D8A0C6EF39F0010ECCEC01F00101FC
:10738000CB2BD8B4CC2B0001D8A4E9D7939281821F
:1073900081A8CDEF39F0EDEF3AF0D896060105A1BE
:1073A000D8860001D8B6F2EF39F00101CC6B010E9E
:1073B000CB6F00010101CB510501F15D0101CC5101
:1073C0000501F2590001D8A0F0EF39F0010ECCEC24
:1073D00001F00101CB2BD8B4CC2B0001D8A4E9D704
:1073E0009394818481A8F7EF39F0EDEF3AF0D0EF74
:1073F0003AF081A8FEEF39F0EDEF3AF0D8960501AA
:10740000E4A9D8860001D8B623EF3AF00101CC6B8D
:10741000010ECB6F00010101CB510501F15D0101AE
:10742000CC510501F2590001D8A021EF3AF0010E2C
:10743000CCEC01F00101CB2BD8B4CC2B0001D8A4AB
:10744000E9D79394818481A828EF3AF0EDEF3AF0E0
:10745000D8960501E4ABD8860001D8B64DEF3AF0D6
:107460000101CC6B010ECB6F00010101CB51050175
:10747000EF5D0101CC510501F0590001D8A04BEF9F
:107480003AF0010ECCEC01F00101CB2BD8B4CC2B9F
:107490000001D8A4E9D79392818281A852EF3AF0F3
:1074A000EDEF3AF0D8960501E4ADD8860001D8B6E4
:1074B00077EF3AF00101CC6B010ECB6F00010101B7
:1074C000CB510501ED5D0101CC510501EE590001E3
:1074D000D8A075EF3AF0010ECCEC01F00101CB2BF6
:1074E000D8B4CC2B0001D8A4E9D79390818081A88F
:1074F0007CEF3AF0EDEF3AF0D8960501E4AFD8868C
:107500000001D8B6A1EF3AF00101CC6B010ECB6FB0
:1075100000010101CB510501EB5D0101CC510501D9
:10752000EC590001D8A09FEF3AF0010ECCEC01F02D
:107530000101CB2BD8B4CC2B0001D8A4E9D7949A65
:10754000828A81A8A6EF3AF0EDEF3AF0D8960601CC
:1075500005A1D8860001D8B6CBEF3AF00101CC6B7B
:10756000010ECB6F00010101CB510501E95D010165
:10757000CC510501EA590001D8A0C9EF3AF0010E3B
:10758000CCEC01F00101CB2BD8B4CC2B0001D8A45A
:10759000E9D79498828881A8D0EF3AF0EDEF3AF0DD
:1075A0000501288DD896060105B7D8860001D8B602
:1075B000DCEF3AF05DEC25F044EF17F00501289D73
:1075C000000144EF17F00501288D000181A8EBEFC1
:1075D0003AF0EDEF3AF044EF17F0BCEC29F044EF4D
:1075E00017F0160EF76E120EF66E01EE2FF0A9ECE4
:1075F00002F0D8A4FFEF3AF0010E0101696F00011B
:10760000160EF76E1A0EF66E01EE2FF0A9EC02F0D0
:10761000D8A419EF3BF00101696B04EEA2F0160E3D
:10762000F76E220EF66E81EC02F0EF6A000165EC57
:107630001DF01200160EF76E380EF66E01EE2FF0EA
:10764000A9EC02F0D8A42DEF3BF006010587010E4E
:107650000101666F00013DEF3BF006010597010156
:10766000666B04EEA2F0160EF76E3C0EF66E81EC21
:1076700002F0EF6A000165EC1DF01200160EF76EC5
:107680004C0EF66E01EE2FF0A9EC02F0D8A44EEFEE
:107690003BF0060105970101666B676B0001160E52
:1076A000F76E520EF66E01EE2FF0A9EC02F0D8A4A0
:1076B00061EF3BF006010587010E0101666F010EC7
:1076C000676F0001120005EECEF011EE2FF0060EEE
:1076D000E6CFEEFFE82EFCD7EF6A04EEA2F0160E1E
:1076E000F76E5A0EF66E81EC02F015EECEF0060E35
:1076F000E75204E0E6CFEEFFE82EFAD7EF6A65EC3A
:107700001DF0120005EE90F015EECEF0060EE752D9
:1077100004E0E6CFEEFFE82EFAD7EF6A82EC2AF01B
:10772000120004EEA2F0160EF76E6C0EF66E81ECEF
:1077300002F011EE2FF0360EE75204E0E6CFEEFF36
:10774000E82EFAD7EF6A65EC1DF001EE2FF084EC1D
:1077500000F00501D66F1FC0D7F50001120004EE3E
:10776000A2F0160EF76E820EF66E81EC02F011EEAC
:107770002FF0360EE75204E0E6CFEEFFE82EFAD700
:10778000EF6A65EC1DF001EE2FF084EC00F00501CE
:10779000D86F1FC0D9F5000112000BEC37F004EED2
:1077A000A2F0160EF76E9A0EF66E81EC02F0020E43
:1077B000016E0501E351CCEC00F0EF6A000165ECCD
:1077C0001DF0120004EEA2F0160EF76EB20EF66E69
:1077D00081EC02F011EE2FF0360EE75204E0E6CF16
:1077E000EEFFE82EFAD72E0EEE6EEF6A65EC1DF076
:1077F00001EE2FF084EC00F00501E36F00011200B0
:1078000004EEA2F0160EF76ECE0EF66E81EC02F0CC
:1078100011EE2FF0360EE75204E0E6CFEEFFE82E31
:10782000FAD7200EEE6E6D0EEE6E730EEE6E2E0E0D
:10783000EE6EEF6A65EC1DF001EE2FF084EC00F0C7
:107840000501E96F1FC0EAF50001120004EEA2F085
:10785000160EF76EE40EF66E81EC02F011EE2FF0CC
:10786000360EE75204E0E6CFEEFFE82EFAD7200E00
:10787000EE6E6D0EEE6E730EEE6E2E0EEE6EEF6A07
:1078800065EC1DF001EE2FF084EC00F00501EB6FCC
:107890001FC0ECF50001120004EEA2F0160EF76E08
:1078A000FA0EF66E81EC02F011EE2FF0360EE75272
:1078B00004E0E6CFEEFFE82EFAD7200EEE6E6D0E56
:1078C000EE6E730EEE6E2E0EEE6EEF6A65EC1DF030
:1078D00001EE2FF084EC00F00501ED6F1FC0EEF516
:1078E0000001120004EEA2F0170EF76E100EF66EF5
:1078F00081EC02F011EE2FF0360EE75204E0E6CFF5
:10790000EEFFE82EFAD7200EEE6E6D0EEE6E730EC1
:10791000EE6E2E0EEE6EEF6A65EC1DF001EE2FF0AE
:1079200084EC00F00501EF6F1FC0F0F500011200BC
:1079300004EEA2F0170EF76E260EF66E81EC02F042
:1079400011EE2FF0360EE75204E0E6CFEEFFE82E00
:10795000FAD7200EEE6E6D0EEE6E730EEE6E2E0EDC
:10796000EE6EEF6A65EC1DF001EE2FF084EC00F096
:107970000501F16F1FC0F2F50001120004EEA2F044
:10798000170EF76E3C0EF66E81EC02F011EE2FF042
:10799000360EE75204E0E6CFEEFFE82EFAD7200ECF
:1079A000EE6E6D0EEE6E730EEE6E2E0EEE6EEF6AD6
:1079B00065EC1DF001EE2FF084EC00F00501F76F8F
:1079C0001FC0F8F50001120004EEA2F0170EF76ECA
:1079D000500EF66E81EC02F011EE2FF0360EE752EB
:1079E00004E0E6CFEEFFE82EFAD7200EEE6E6D0E25
:1079F000EE6E730EEE6E2E0EEE6EEF6A65EC1DF0FF
:107A000001EE2FF084EC00F00501F96F1FC0FAF5CC
:107A10000001120004EEA2F0170EF76E640EF66E6F
:107A200081EC02F011EE2FF0360EE75204E0E6CFC3
:107A3000EEFFE82EFAD7200EEE6E6D0EEE6E730E90
:107A4000EE6E2E0EEE6EEF6A65EC1DF001EE2FF07D
:107A500084EC00F00501FB6F1FC0FCF50001120073
:107A600004EEA2F0170EF76E780EF66E81EC02F0BF
:107A700011EE2FF0360EE75204E0E6CFEEFFE82ECF
:107A8000FAD7200EEE6E6D0EEE6E730EEE6E2E0EAB
:107A9000EE6EEF6A65EC1DF001EE2FF084EC00F065
:107AA0000501FD6F1FC0FEF50001120004EEA2F0FB
:107AB000170EF76E8C0EF66E81EC02F011EE2FF0C1
:107AC000360EE75204E0E6CFEEFFE82EFAD7200E9E
:107AD000EE6E6D0EEE6E730EEE6E2E0EEE6EEF6AA5
:107AE00065EC1DF001EE2FF084EC00F00501FF6F56
:107AF0001FC000F600011200310E01012F5D0001D0
:107B0000D8A48AEF3DF00501E48901EE9EF0310E24
:107B1000EE6EEF6A0001320E01012F5D0001D8A464
:107B200099EF3DF00501E48B01EE9EF0320EEE6E12
:107B3000EF6A0001330E01012F5D0001D8A4A8EF08
:107B40003DF00501E48D01EE9EF0330EEE6EEF6A1E
:107B50000001340E01012F5D0001D8A4B7EF3DF004
:107B60000501E48F01EE9EF0340EEE6EEF6A000127
:107B7000350E01012F5D0001D8A4C6EF3DF00601CE
:107B8000058101EE9EF0350EEE6EEF6A000104EE07
:107B9000A2F0170EF76EA00EF66E81EC02F011EE59
:107BA0009EF0140EE75204E0E6CFEEFFE82EFAD77F
:107BB000170EF76EA80EF66E81EC02F0EF6A65EC18
:107BC0001DF01200310E01012F5D0001D8A4F0EF6D
:107BD0003DF00501E49901EE9EF0310EEE6EEF6A84
:107BE0000001320E01012F5D0001D8A4FFEF3DF02E
:107BF0000501E49B01EE9EF0320EEE6EEF6A00018D
:107C0000330E01012F5D0001D8A40EEF3EF00501F7
:107C1000E49D01EE9EF0330EEE6EEF6A0001340E2D
:107C200001012F5D0001D8A41DEF3EF00501E49F86
:107C300001EE9EF0340EEE6EEF6A0001350E01018A
:107C40002F5D0001D8A42CEF3EF00601059101EE56
:107C50009EF0350EEE6EEF6A000104EEA2F0170EF4
:107C6000F76EB20EF66E81EC02F011EE9EF0140E7D
:107C7000E75204E0E6CFEEFFE82EFAD7170EF76ED4
:107C8000BA0EF66E81EC02F0EF6A65EC1DF01200A0
:107C9000170EF76EC40EF66E01EE2FF0A9EC02F08F
:107CA000D8A454EF3EF08288170EF76EC80EF66E19
:107CB00001EE2FF0A9EC02F0D8A460EF3EF082981C
:107CC00082A86EEF3EF004EEA2F0170EF76ECC0E17
:107CD000F66E81EC02F0EF6A65EC1DF082B87CEF85
:107CE0003EF004EEA2F0170EF76EDE0EF66E81EC9B
:107CF00002F0EF6A65EC1DF01200170EF76EF00E41
:107D0000F66E01EE2FF0A9EC02F0D8A489EF3EF058
:107D1000828A170EF76EF40EF66E01EE2FF0A9ECC4
:107D200002F0D8A495EF3EF0829A82AAA3EF3EF02B
:107D300004EEA2F0170EF76EF80EF66E81EC02F06C
:107D4000EF6A65EC1DF082BAB1EF3EF004EEA2F0EE
:107D5000180EF76E0A0EF66E81EC02F0EF6A65EC13
:107D60001DF01200180EF76E1C0EF66E01EE2FF0CD
:107D7000A9EC02F0D8A4BEEF3EF08180180EF76E99
:107D8000200EF66E01EE2FF0A9EC02F0D8A4CAEF97
:107D90003EF0819081A0D8EF3EF004EEA2F0180EE4
:107DA000F76E240EF66E81EC02F0EF6A65EC1DF0C2
:107DB00081B0E6EF3EF004EEA2F0180EF76E360E3C
:107DC000F66E81EC02F0EF6A65EC1DF01200180E01
:107DD000F76E480EF66E01EE2FF0A9EC02F0D8A473
:107DE000F3EF3EF08182180EF76E4C0EF66E01EE48
:107DF0002FF0A9EC02F0D8A4FFEF3EF0819281A20F
:107E00000DEF3FF004EEA2F0180EF76E500EF66E76
:107E100081EC02F0EF6A65EC1DF081B21BEF3FF0E0
:107E200004EEA2F0180EF76E620EF66E81EC02F010
:107E3000EF6A65EC1DF01200180EF76E740EF66E08
:107E400001EE2FF0A9EC02F0D8A428EF3FF08184D6
:107E5000180EF76E780EF66E01EE2FF0A9EC02F018
:107E6000D8A434EF3FF0819481A442EF3FF004EEB8
:107E7000A2F0180EF76E7C0EF66E81EC02F0EF6A3F
:107E800065EC1DF081B450EF3FF004EEA2F0180E47
:107E9000F76E8E0EF66E81EC02F0EF6A65EC1DF067
:107EA0001200120012001200180EF76EA00EF66EED
:107EB00001EE2FF0A9EC02F0D8A461EF3FF006012B
:107EC000078F0001180EF76EA40EF66E01EE2FF06C
:107ED000A9EC02F0D8A46FEF3FF00601079F000164
:107EE000D896060107AFD8860001D8B683EF3FF0D9
:107EF00004EEA2F0180EF76EA80EF66E81EC02F0FA
:107F0000EF6A65EC1DF0D896060107BFD886000120
:107F1000D8B696EF3FF004EEA2F0180EF76EB80E4A
:107F2000F66E81EC02F0EF6A65EC1DF00601058D3E
:107F300000011200180EF76ECA0EF66E01EE2FF059
:107F4000A9EC02F0D8A4A7EF3FF0060108810001D8
:107F5000180EF76ECE0EF66E01EE2FF0A9EC02F0C1
:107F6000D8A4B5EF3FF0060108910001D8960601AC
:107F700008A1D8860001D8B6C9EF3FF004EEA2F000
:107F8000180EF76ED20EF66E81EC02F0EF6A65EC19
:107F90001DF0D896060108B1D8860001D8B6DCEFEE
:107FA0003FF004EEA2F0180EF76EE20EF66E81ECD2
:107FB00002F0EF6A65EC1DF00601058D000112006C
:107FC000180EF76EF40EF66E01EE2FF0A9EC02F02B
:107FD000D8A4EDEF3FF0060108830001180EF76EFC
:107FE000F80EF66E01EE2FF0A9EC02F0D8A4FBEF2C
:107FF0003FF0060108930001D896060108A3D88631
:108000000001D8B60FEF40F004EEA2F0180EF76EA4
:10801000FC0EF66E81EC02F0EF6A65EC1DF0D8966E
:10802000060108B3D8860001D8B622EF40F004EE6E
:10803000A2F0190EF76E0C0EF66E81EC02F0EF6AEC
:1080400065EC1DF00601058D0001120004EEA2F0A2
:10805000190EF76E1E0EF66E81EC02F0EF6A65ECFB
:108060001DF0010E0501E36F010EE16FEA6B010ED9
:10807000E96FEC6B640EEB6FEE6B640EED6FF06B03
:10808000640EEF6FF26B640EF16FF46B640EF36FBE
:10809000F66B640EF56FF86B010EF76FFA6B640EFA
:1080A000F96FFC6B640EFB6FFE6B640EFD6F0601D7
:1080B000006B640E0501FF6F0601026B640E016F19
:1080C000046B640E036F0589058B140E05018E6F1A
:1080D000756BCD0E796FCC0E786F4C0E776F7C0E72
:1080E000766F060105950501486B476B466B456B3E
:1080F0004C6B4B6B4A6B496B506B4F6B4E6B4D6BC4
:10810000546B536B526B516B010167530001D8A440
:108110008CEF40F08CEC47F00101696B666B060157
:1081200005970501236B586B576B566B556B5C6B52
:108130005B6B5A6B596B606B5F6B5E6B5D6B646BFB
:10814000636B626B616B686B676B700E666F830E3F
:10815000656F6C6B6B6B700E6A6F830E696F706B03
:108160006F6B700E6E6F830E6D6F746B736B700E32
:10817000726F830E716F0401A16B01016A6B0001C4
:108180001200010E0501D56FAA6AA96AD551A6ECA5
:1081900001F00A0ECCEC01F0AA6A020EA96ED651CB
:1081A000A6EC01F0D751A6EC01F00A0ECCEC01F0E0
:1081B000AA6A040EA96ED851A6EC01F0D951A6EC1A
:1081C00001F00A0ECCEC01F0AA6A060EA96EE3518A
:1081D000A6EC01F00A0ECCEC01F0AA6A0A0EA96E18
:1081E000000EA6EC01F0AA6A140EA96EE951A6ECE5
:1081F00001F0EA51A6EC01F00A0ECCEC01F0AA6AFB
:10820000160EA96EEB51A6EC01F0EC51A6EC01F0B4
:108210000A0ECCEC01F0AA6A180EA96EED51A6EC7C
:1082200001F0EE51A6EC01F00A0ECCEC01F0AA6AC6
:108230001A0EA96EEF51A6EC01F0F051A6EC01F078
:108240000A0ECCEC01F0AA6A1C0EA96EF151A6EC44
:1082500001F0F251A6EC01F00A0ECCEC01F0AA6A92
:108260001E0EA96EF351A6EC01F0F451A6EC01F03C
:108270000A0ECCEC01F0AA6A200EA96EF551A6EC0C
:1082800001F0F651A6EC01F00A0ECCEC01F0AA6A5E
:10829000280EA96EF751A6EC01F0F851A6EC01F0FA
:1082A0000A0ECCEC01F0AA6A2A0EA96EF951A6ECCE
:1082B00001F0FA51A6EC01F00A0ECCEC01F0AA6A2A
:1082C0002C0EA96EFB51A6EC01F0FC51A6EC01F0BE
:1082D0000A0ECCEC01F0AA6A2E0EA96EFD51A6EC96
:1082E00001F0FE51A6EC01F00A0ECCEC01F0AA6AF6
:1082F000300EA96EFF51A6EC01F006010051A6EC6C
:1083000001F00A0ECCEC01F0AA6A320EA96E0151FE
:10831000A6EC01F00251A6EC01F00A0ECCEC01F043
:10832000AA6A340EA96E0351A6EC01F00451A6EC22
:1083300001F00A0ECCEC01F0AA6A3C0EA96EE86AC4
:1083400005B9010EA6EC01F00A0ECCEC01F0AA6A08
:108350003E0EA96EE86A05BB010EA6EC01F00A0EFE
:10836000CCEC01F0AA6A400EA96E0401A151A6EC62
:1083700001F00A0ECCEC01F0AA6A410EA96E05EEDE
:10838000CEF0EE5003E0A6EC01F0FBD70A0ECCECE9
:1083900001F001EEC8F015EECEF0010EF36E010E05
:1083A00089EC02F0EF6AAA6A410EA96E01EEC8F0EC
:1083B000EE5003E0A6EC01F0FBD70A0ECCEC01F086
:1083C00001EEC8F015EECEF0020EF36E010E89EC50
:1083D00002F0EF6AAA6A420EA96E01EEC8F0EE50F2
:1083E00003E0A6EC01F0FBD70A0ECCEC01F001EEA5
:1083F000C8F015EECEF0030EF36E010E89EC02F01C
:10840000EF6AAA6A430EA96E01EEC8F0EE5003E0CF
:10841000A6EC01F0FBD70A0ECCEC01F001EEC8F09F
:1084200015EECEF0040EF36E010E89EC02F0EF6A49
:10843000AA6A440EA96E01EEC8F0EE5003E0A6EC65
:1084400001F0FBD70A0ECCEC01F001EEC8F015EEFE
:10845000CEF0050EF36E010E89EC02F0EF6AAA6A07
:10846000450EA96E01EEC8F0EE5003E0A6EC01F057
:10847000FBD70A0ECCEC01F001EEC8F015EECEF001
:10848000060EF36E010E89EC02F0EF6AAA6A460E40
:10849000A96E01EEC8F0EE5003E0A6EC01F0FBD7A8
:1084A0000A0ECCEC01F0AA6A500EA96EE86A05012A
:1084B000E4B9010EA6EC01F00A0ECCEC01F0AA6AB8
:1084C000510EA96EE86AE4BB010EA6EC01F00A0E9B
:1084D000CCEC01F0AA6A520EA96EE86AE4BD010E66
:1084E000A6EC01F00A0ECCEC01F0AA6A530EA96EBC
:1084F000E86AE4BF010EA6EC01F00A0ECCEC01F034
:10850000AA6A540EA96EE86A060105B1010EA6EC2E
:1085100001F00A0ECCEC01F0AA6A550EA96E050115
:108520008E51A6EC01F00A0ECCEC01F0AA6A560EB0
:10853000A96E7551A6EC01F00A0ECCEC01F0AA6A06
:10854000570EA96E7651A6EC01F07751A6EC01F01A
:108550007851A6EC01F07951A6EC01F00A0ECCECB2
:1085600001F0AA6A5B0EA96EE86A060105B7010E62
:10857000A6EC01F00A0ECCEC01F0AA6A5C0EA96E22
:1085800005014551A6EC01F04651A6EC01F047511A
:10859000A6EC01F04851A6EC01F00A0ECCEC01F07B
:1085A000AA6A600EA96E4951A6EC01F04A51A6ECE8
:1085B00001F04B51A6EC01F04C51A6EC01F00A0E73
:1085C000CCEC01F0AA6A640EA96E4D51A6EC01F044
:1085D0004E51A6EC01F04F51A6EC01F05051A6EC23
:1085E00001F00A0ECCEC01F0AA6A680EA96E515196
:1085F000A6EC01F05251A6EC01F05351A6EC01F0AB
:108600005451A6EC01F00A0ECCEC01F0AA6A6C0EF3
:10861000A96E01016651A6EC01F00A0ECCEC01F046
:10862000AA6A6D0EA96E6751A6EC01F00A0ECCEC99
:1086300001F0AA6A6E0EA96E6951A6EC01F00A0E4D
:10864000CCEC01F0AA6A6F0EA96E05015551A6EC9B
:1086500001F05651A6EC01F05751A6EC01F058512B
:10866000A6EC01F00A0ECCEC01F0AA6A730EA96E1A
:108670005951A6EC01F05A51A6EC01F05B51A6EC61
:1086800001F05C51A6EC01F00A0ECCEC01F0AA6AF4
:10869000770EA96E5D51A6EC01F05E51A6EC01F0DB
:1086A0005F51A6EC01F06051A6EC01F00A0ECCEC93
:1086B00001F0AA6A7B0EA96E6151A6EC01F062512D
:1086C000A6EC01F06351A6EC01F06451A6EC01F0B8
:1086D0000A0ECCEC01F0AA6A7F0EA96E6551A6ECD9
:1086E00001F06651A6EC01F06751A6EC01F068516B
:1086F000A6EC01F00A0ECCEC01F0AA6A830EA96E7A
:108700006951A6EC01F06A51A6EC01F06B51A6ECA0
:1087100001F06C51A6EC01F00A0ECCEC01F0AA6A53
:10872000870EA96E6D51A6EC01F06E51A6EC01F01A
:108730006F51A6EC01F07051A6EC01F00A0ECCECE2
:1087400001F0AA6A8B0EA96E7151A6EC01F072516C
:10875000A6EC01F07351A6EC01F07451A6EC01F007
:108760000A0ECCEC01F0AA6A8F0EA96E01016A51C3
:10877000A6EC01F00A0ECCEC01F0AA6A900EA96EEC
:1087800005012351A6EC01F00A0ECCEC01F004EE39
:10879000A2F0190EF76E460EF66E81EC02F0EF6A4B
:1087A000000165EC1DF01200000E9DEC01F00501CA
:1087B000D56F020E9DEC01F0D66F9FEC01F0D76FE4
:1087C000040E9DEC01F0D86F9FEC01F0D96F060EFE
:1087D0009DEC01F0E36F0A0E9DEC01F0E16FE129E1
:1087E000E26F140E9DEC01F0E96F9FEC01F0EA6F6F
:1087F000160E9DEC01F0EB6F9FEC01F0EC6F180E84
:108800009DEC01F0ED6F9FEC01F0EE6F1A0E9DEC08
:1088100001F0EF6F9FEC01F0F06F1C0E9DEC01F08A
:10882000F16F9FEC01F0F26F1E0E9DEC01F0F36F03
:108830009FEC01F0F46F200E9DEC01F0F56F9FECC2
:1088400001F0F66F280E9DEC01F0F76F9FEC01F040
:10885000F86F2A0E9DEC01F0F96F9FEC01F0FA6FB2
:108860002C0E9DEC01F0FB6F9FEC01F0FC6F2E0EC7
:108870009DEC01F0FD6F9FEC01F0FE6F300E9DEC62
:1088800001F0FF6F9FEC01F00601006F320E9DECCE
:1088900001F0016F9FEC01F0026F340E9DEC01F0CE
:1088A000036F9FEC01F0046F3C0E9DEC01F0058915
:1088B000E8A005993E0E9DEC01F0058BE8A0059B14
:1088C000400E9DEC01F00401A16F500E9DEC01F0F3
:1088D0000501E489E8A0E499510E9DEC01F0E48BD8
:1088E000E8A0E49B520E9DEC01F0E48DE8A0E49D2D
:1088F000530E9DEC01F0E48FE8A0E49F540E9DEC34
:1089000001F006010581E8A00591550E9DEC01F0EE
:1089100005018E6F560E9DEC01F0756F570E9DECA4
:1089200001F0766F9FEC01F0776F9FEC01F0786FAC
:108930009FEC01F0796F5B0E9DEC01F0060105875D
:10894000E8A005975C0E9DEC01F00501456F9FECDA
:1089500001F0466F9FEC01F0476F9FEC01F0486F0C
:10896000600E9DEC01F0496F9FEC01F04A6F9FECA7
:1089700001F04B6F9FEC01F04C6F640E9DEC01F029
:108980004D6F9FEC01F04E6F9FEC01F04F6F9FEC2D
:1089900001F0506F680E9DEC01F0516F9FEC01F0FB
:1089A000526F9FEC01F0536F9FEC01F0546F6C0E0F
:1089B0009DEC01F00101666F6D0E9DEC01F0676F9B
:1089C0006E0E9DEC01F0696F6F0E9DEC01F00501DC
:1089D000556F9FEC01F0566F9FEC01F0576F9FECC5
:1089E00001F0586F730E9DEC01F0596F9FEC01F090
:1089F0005A6F9FEC01F05B6F9FEC01F05C6F770E9C
:108A00009DEC01F05D6F9FEC01F05E6F9FEC01F05B
:108A10005F6F9FEC01F0606F7B0E9DEC01F0616F6A
:108A20009FEC01F0626F9FEC01F0636F9FEC01F02F
:108A3000646F7F0E9DEC01F0656F9FEC01F0666F37
:108A40009FEC01F0676F9FEC01F0686F830E9DEC67
:108A500001F0696F9FEC01F06A6F9FEC01F06B6FA2
:108A60009FEC01F06C6F870E9DEC01F06D6F9FEC39
:108A700001F06E6F9FEC01F06F6F9FEC01F0706F73
:108A80008B0E9DEC01F0716F9FEC01F0726F9FEC0B
:108A900001F0736F9FEC01F0746F8F0E9DEC01F08D
:108AA00001016A6F900E9DEC01F00501236F130E1A
:108AB000EA5D0001D8A06BEF45F0D8A467EF45F060
:108AC000890E0501E95D0001D8A06BEF45F00501B5
:108AD000EA6B320EE96F0001010169530001D8A46D
:108AE00074EF45F08CEC47F0010169530001D8A404
:108AF00085EF45F004EEA2F0190EF76E6C0EF66EDF
:108B000081EC02F0EF6A65EC1DF0120004EEA2F0B9
:108B1000190EF76E940EF66E81EC02F0EF6A65ECBA
:108B20001DF004EEA2F0190EF76ED00EF66E81EC79
:108B300002F0EF6A65EC1DF004EEA2F01A0EF76E7B
:108B4000220EF66E81EC02F0EF6A65EC1DF004EE89
:108B5000A2F01A0EF76E740EF66E81EC02F0EF6A58
:108B600065EC1DF004EEA2F01A0EF76EBC0EF66E68
:108B700081EC02F0EF6A65EC1DF004EEA2F01B0E32
:108B8000F76E040EF66E81EC02F0EF6A65EC1DF0F4
:108B900004EEA2F01B0EF76E420EF66E81EC02F0B0
:108BA000EF6A65EC1DF004EEA2F01B0EF76E800E6E
:108BB000F66E81EC02F0EF6A65EC1DF004EEA2F0B7
:108BC0001B0EF76EA80EF66E81EC02F0EF6A65ECF4
:108BD0001DF004EEA2F01B0EF76ED20EF66E81ECC5
:108BE00002F0EF6A65EC1DF004EEA2F01C0EF76EC9
:108BF000100EF66E81EC02F0EF6A65EC1DF004EEEB
:108C0000A2F01C0EF76E400EF66E81EC02F0EF6AD9
:108C100065EC1DF004EEA2F01C0EF76E740EF66EFD
:108C200081EC02F0EF6A65EC1DF004EEA2F01C0E80
:108C3000F76EAA0EF66E81EC02F0EF6A65EC1DF09D
:108C400004EEA2F01C0EF76EDE0EF66E81EC02F062
:108C5000EF6A65EC1DF004EEA2F01D0EF76E260E15
:108C6000F66E81EC02F0EF6A65EC1DF004EEA2F006
:108C70001D0EF76E4A0EF66E81EC02F0EF6A65EC9F
:108C80001DF004EEA2F01D0EF76E720EF66E81EC72
:108C900002F0EF6A65EC1DF004EEA2F01D0EF76E17
:108CA0009A0EF66E81EC02F0EF6A65EC1DF004EEB0
:108CB000A2F01D0EF76ED80EF66E81EC02F0EF6A90
:108CC00065EC1DF004EEA2F01E0EF76E380EF66E87
:108CD00081EC02F0EF6A65EC1DF004EEA2F01E0ECE
:108CE000F76E800EF66E81EC02F0EF6A65EC1DF017
:108CF00004EEA2F01E0EF76ECA0EF66E81EC02F0C4
:108D0000EF6A65EC1DF004EEA2F01E0EF76EFA0E8F
:108D1000F66E81EC02F0EF6A65EC1DF004EEA2F055
:108D20001F0EF76E380EF66E81EC02F0EF6A65ECFE
:108D30001DF004EEA2F01F0EF76E980EF66E81EC99
:108D400002F0EF6A65EC1DF004EEA2F01F0EF76E64
:108D5000D00EF66E81EC02F0EF6A65EC1DF004EEC9
:108D6000A2F0200EF76E400EF66E81EC02F0EF6A74
:108D700065EC1DF004EEA2F0200EF76E8A0EF66E82
:108D800081EC02F0EF6A65EC1DF004EEA2F0200E1B
:108D9000F76EC80EF66E81EC02F0EF6A65EC1DF01E
:108DA00004EEA2F0210EF76E1A0EF66E81EC02F0C0
:108DB000EF6A65EC1DF004EEA2F0210EF76E700E66
:108DC000F66E81EC02F0EF6A65EC1DF004EEA2F0A5
:108DD000210EF76EB40EF66E81EC02F0EF6A65ECD0
:108DE0001DF004EEA2F0210EF76EFA0EF66E81EC85
:108DF00002F0EF6A65EC1DF004EEA2F0220EF76EB1
:108E0000380EF66E81EC02F0EF6A65EC1DF004EEB0
:108E1000A2F0220EF76E840EF66E81EC02F0EF6A7D
:108E200065EC1DF004EEA2F0220EF76EC20EF66E97
:108E300081EC02F0EF6A65EC1DF004EEA2F0230E67
:108E4000F76E0A0EF66E81EC02F0EF6A65EC1DF02B
:108E500004EEA2F0230EF76E4C0EF66E81EC02F0DB
:108E6000EF6A65EC1DF004EEA2F0230EF76E800EA3
:108E7000F66E81EC02F0EF6A65EC1DF004EEA2F0F4
:108E8000230EF76EB80EF66E81EC02F0EF6A65EC19
:108E90001DF004EEA2F0230EF76EF60EF66E81ECD6
:108EA00002F0EF6A65EC1DF004EEA2F0240EF76EFE
:108EB000280EF66E81EC02F0EF6A65EC1DF004EE10
:108EC000A2F0240EF76E5A0EF66E81EC02F0EF6AF5
:108ED00065EC1DF004EEA2F0240EF76E980EF66E0F
:108EE00081EC02F0EF6A65EC1DF004EEA2F0240EB6
:108EF000F76EC40EF66E81EC02F0EF6A65EC1DF0C1
:108F000004EEA2F0240EF76EF20EF66E81EC02F083
:108F1000EF6A65EC1DF0120004EEA2F0250EF76E6C
:108F2000360EF66E81EC02F0EF6A65EC1DF001EE94
:108F30006BF0020E016E0501D551CCEC00F0EF6A2A
:108F400004EEA2F0250EF76E5E0EF66E81EC02F0D6
:108F500011EE6BF0320EE75204E0E6CFEEFFE82EA2
:108F6000FAD7EF6A000165EC1DF001EE6BF015EE2B
:108F7000DAF0060EE75204E0E6CFEEFFE82EFAD76D
:108F8000EF6A04EEA2F0250EF76E6E0EF66E81EC1F
:108F900002F011EE6BF0320EE75204E0E6CFEEFF86
:108FA000E82EFAD7EF6A65EC1DF001EE6BF0020EC9
:108FB000016E066AD7C51FF0D6C51EF0CFEC00F0D3
:108FC000EF6A04EEA2F0250EF76E7E0EF66E81ECCF
:108FD00002F011EE6BF0320EE75204E0E6CFEEFF46
:108FE000E82EFAD7EF6A65EC1DF001EE6BF0020E89
:108FF000016E066AD9C51FF0D8C51EF0CFEC00F08F
:10900000EF6A04EEA2F0250EF76E8E0EF66E81EC7E
:1090100002F011EE6BF0320EE75204E0E6CFEEFF05
:10902000E82EFAD7EF6A65EC1DF001EE6BF0020E48
:10903000016E0501E351CCEC00F0EF6A04EEA2F002
:10904000250EF76E9E0EF66E81EC02F011EE6BF0BF
:10905000320EE75204E0E6CFEEFFE82EFAD7EF6AD1
:10906000000165EC1DF001EE6BF0020E016E066A68
:10907000EAC51FF0E9C51EF0CFEC00F0EF6A04EE80
:10908000A2F0250EF76EAE0EF66E81EC02F011EE38
:109090006BF0320EE75204E0E6CFEEFFE82EFAD78F
:1090A000EF6A65EC1DF001EE6BF0020E016E066AD0
:1090B000ECC51FF0EBC51EF0CFEC00F0EF6A04EE3C
:1090C000A2F0250EF76EBE0EF66E81EC02F011EEE8
:1090D0006BF0320EE75204E0E6CFEEFFE82EFAD74F
:1090E000EF6A65EC1DF001EE6BF0020E016E066A90
:1090F000EEC51FF0EDC51EF0CFEC00F0EF6A04EEF8
:10910000A2F0250EF76ECE0EF66E81EC02F011EE97
:109110006BF0320EE75204E0E6CFEEFFE82EFAD70E
:10912000EF6A65EC1DF001EE6BF0020E016E066A4F
:10913000F0C51FF0EFC51EF0CFEC00F0EF6A04EEB3
:10914000A2F0250EF76EDE0EF66E81EC02F011EE47
:109150006BF0320EE75204E0E6CFEEFFE82EFAD7CE
:10916000EF6A65EC1DF001EE6BF0020E016E066A0F
:10917000F2C51FF0F1C51EF0CFEC00F0EF6A04EE6F
:10918000A2F0250EF76EEE0EF66E81EC02F011EEF7
:109190006BF0320EE75204E0E6CFEEFFE82EFAD78E
:1091A000EF6A65EC1DF001EE6BF0020E016E066ACF
:1091B000F8C51FF0F7C51EF0CFEC00F0EF6A04EE23
:1091C000A2F0250EF76EFE0EF66E81EC02F011EEA7
:1091D0006BF0320EE75204E0E6CFEEFFE82EFAD74E
:1091E000EF6A65EC1DF001EE6BF0020E016E066A8F
:1091F000FAC51FF0F9C51EF0CFEC00F0EF6A04EEDF
:10920000A2F0260EF76E0E0EF66E81EC02F011EE55
:109210006BF0320EE75204E0E6CFEEFFE82EFAD70D
:10922000EF6A65EC1DF001EE6BF0020E016E066A4E
:10923000FCC51FF0FBC51EF0CFEC00F0EF6A04EE9A
:10924000A2F0260EF76E1E0EF66E81EC02F011EE05
:109250006BF0320EE75204E0E6CFEEFFE82EFAD7CD
:10926000EF6A65EC1DF001EE6BF0020E016E066A0E
:10927000FEC51FF0FDC51EF0CFEC00F0EF6A04EE56
:10928000A2F0260EF76E2E0EF66E81EC02F011EEB5
:109290006BF0320EE75204E0E6CFEEFFE82EFAD78D
:1092A000EF6A65EC1DF001EE6BF0020E016E066ACE
:1092B00000C61FF0FFC51EF0CFEC00F0EF6A04EE11
:1092C000A2F0260EF76E3E0EF66E81EC02F011EE65
:1092D0006BF0320EE75204E0E6CFEEFFE82EFAD74D
:1092E000EF6A65EC1DF0D8960501E4A9D886000167
:1092F000D8B686EF49F001EE9EF0260EF76E4E0EC0
:10930000F66E81EC02F0EF6A8FEF49F001EE9EF00D
:10931000260EF76E580EF66E81EC02F0EF6A04EE40
:10932000A2F0260EF76E640EF66E81EC02F011EEDE
:109330009EF0140EE75204E0E6CFEEFFE82EFAD7D7
:10934000EF6A65EC1DF0D8960501E4ABD886000104
:10935000D8B6B6EF49F001EE9EF0260EF76E720E0B
:10936000F66E81EC02F0EF6ABFEF49F001EE9EF07D
:10937000260EF76E7C0EF66E81EC02F0EF6A04EEBC
:10938000A2F0260EF76E880EF66E81EC02F011EE5A
:109390009EF0140EE75204E0E6CFEEFFE82EFAD777
:1093A000EF6A65EC1DF0D8960501E4ADD8860001A2
:1093B000D8B6E6EF49F001EE9EF0260EF76E960E57
:1093C000F66E81EC02F0EF6AEFEF49F001EE9EF0ED
:1093D000260EF76EA00EF66E81EC02F0EF6A04EE38
:1093E000A2F0260EF76EAC0EF66E81EC02F011EED6
:1093F0009EF0140EE75204E0E6CFEEFFE82EFAD717
:10940000EF6A65EC1DF0D8960501E4AFD88600013F
:10941000D8B616EF4AF001EE9EF0260EF76EBA0EA1
:10942000F66E81EC02F0EF6A1FEF4AF001EE9EF05B
:10943000260EF76EC40EF66E81EC02F0EF6A04EEB3
:10944000A2F0260EF76ED00EF66E81EC02F011EE51
:109450009EF0140EE75204E0E6CFEEFFE82EFAD7B6
:10946000EF6A65EC1DF0D896060105A1D8860001CB
:10947000D8B646EF4AF001EE9EF0260EF76EDE0EED
:10948000F66E81EC02F0EF6A4FEF4AF001EE9EF0CB
:10949000260EF76EE80EF66E81EC02F0EF6A04EE2F
:1094A000A2F0260EF76EF40EF66E81EC02F011EECD
:1094B0009EF0140EE75204E0E6CFEEFFE82EFAD756
:1094C000EF6A65EC1DF0D896060105A9D886000163
:1094D000D8B678EF4AF004EEA2F0270EF76E020E2F
:1094E000F66E81EC02F0EF6A65EC1DF083EF4AF056
:1094F00004EEA2F0270EF76E180EF66E81EC02F065
:10950000EF6A65EC1DF0D896060105ABD886000120
:10951000D8B698EF4AF004EEA2F0270EF76E300EA0
:10952000F66E81EC02F0EF6A65EC1DF0A3EF4AF0F5
:1095300004EEA2F0270EF76E460EF66E81EC02F0F6
:10954000EF6A65EC1DF004EEA2F0270EF76E5E0EDA
:10955000F66E81EC02F0020E016E05018E51CCEC2C
:1095600000F0EF6A000165EC1DF005017553000184
:10957000D8A4C4EF4AF004EEA2F0270EF76E6E0EE8
:10958000F66E81EC02F0EF6A010E0501755D0001D7
:10959000D8A4D4EF4AF004EEA2F0270EF76E860EA0
:1095A000F66E81EC02F0EF6A020E0501755D0001B6
:1095B000D8A4F1EF4AF004EEA2F0270EF76EAA0E3F
:1095C000F66E81EC02F0020E016E79C52DF078C5C1
:1095D0002CF077C52BF076C52AF0030EFEEC00F0D8
:1095E000EF6A01016A530001D8A402EF4BF004EEC8
:1095F000A2F0270EF76EC40EF66E81EC02F0EF6A51
:1096000065EC1DF0010E01016A5D0001D8A414EFA4
:109610004BF004EEA2F0270EF76ED80EF66E81EC3A
:1096200002F0EF6A65EC1DF001EE6BF0020E016EC8
:1096300058C52DF057C52CF056C52BF055C52AF04E
:10964000030EFEEC00F0EF6A04EEA2F0270EF76EB8
:10965000EA0EF66E81EC02F011EE6BF0320EE7527C
:1096600004E0E6CFEEFFE82EFAD7EF6A65EC1DF0D6
:1096700001EE6BF0020E016E68C52DF067C52CF08F
:1096800066C52BF065C52AF0030EFEEC00F0EF6A0C
:1096900004EEA2F0270EF76EFA0EF66E81EC02F0E1
:1096A00011EE6BF0320EE75204E0E6CFEEFFE82E4B
:1096B000FAD7EF6A65EC1DF001EE6BF0020E016E59
:1096C00048C52DF047C52CF046C52BF045C52AF0FE
:1096D000030EFEEC00F0EF6A04EEA2F0280EF76E27
:1096E0000A0EF66E81EC02F011EE6BF0320EE752CC
:1096F00004E0E6CFEEFFE82EFAD7EF6A65EC1DF046
:1097000001EE6BF0020E016E5CC52DF05BC52CF016
:109710005AC52BF059C52AF0030EFEEC00F0EF6A93
:1097200004EEA2F0280EF76E1A0EF66E81EC02F02F
:1097300011EE6BF0320EE75204E0E6CFEEFFE82EBA
:10974000FAD7EF6A65EC1DF001EE6BF0020E016EC8
:109750006CC52DF06BC52CF06AC52BF069C52AF0DD
:10976000030EFEEC00F0EF6A04EEA2F0280EF76E96
:109770002A0EF66E81EC02F011EE6BF0320EE7521B
:1097800004E0E6CFEEFFE82EFAD7EF6A65EC1DF0B5
:1097900001EE6BF0020E016E4CC52DF04BC52CF0A6
:1097A0004AC52BF049C52AF0030EFEEC00F0EF6A23
:1097B00004EEA2F0280EF76E3A0EF66E81EC02F07F
:1097C00011EE6BF0320EE75204E0E6CFEEFFE82E2A
:1097D000FAD7EF6A65EC1DF001EE6BF0020E016E38
:1097E00060C52DF05FC52CF05EC52BF05DC52AF07D
:1097F000030EFEEC00F0EF6A04EEA2F0280EF76E06
:109800004A0EF66E81EC02F011EE6BF0320EE7526A
:1098100004E0E6CFEEFFE82EFAD7EF6A65EC1DF024
:1098200001EE6BF0020E016E70C52DF06FC52CF0CD
:109830006EC52BF06DC52AF0030EFEEC00F0EF6A4A
:1098400004EEA2F0280EF76E5A0EF66E81EC02F0CE
:1098500011EE6BF0320EE75204E0E6CFEEFFE82E99
:10986000FAD7EF6A65EC1DF001EE6BF0020E016EA7
:1098700050C52DF04FC52CF04EC52BF04DC52AF02C
:10988000030EFEEC00F0EF6A04EEA2F0280EF76E75
:109890006A0EF66E81EC02F011EE6BF0320EE752BA
:1098A00004E0E6CFEEFFE82EFAD7EF6A65EC1DF094
:1098B00001EE6BF0020E016E64C52DF063C52CF055
:1098C00062C52BF061C52AF0030EFEEC00F0EF6AD2
:1098D00004EEA2F0280EF76E7A0EF66E81EC02F01E
:1098E00011EE6BF0320EE75204E0E6CFEEFFE82E09
:1098F000FAD7EF6A65EC1DF001EE6BF0020E016E17
:1099000074C52DF073C52CF072C52BF071C52AF00B
:10991000030EFEEC00F0EF6A04EEA2F0280EF76EE4
:109920008A0EF66E81EC02F011EE6BF0320EE75209
:1099300004E0E6CFEEFFE82EFAD7EF6A65EC1DF003
:1099400001EE6BF0020E016E54C52DF053C52CF0E4
:1099500052C52BF051C52AF0030EFEEC00F0EF6A61
:1099600004EEA2F0280EF76E9A0EF66E81EC02F06D
:1099700011EE6BF0320EE75204E0E6CFEEFFE82E78
:10998000FAD7EF6A65EC1DF0050123530001D8A456
:10999000D5EF4CF004EEA2F0280EF76EAA0EF66E8C
:1099A00081EC02F0EF6A65EC1DF0010E0501235D0C
:1099B0000001D8A4E7EF4CF004EEA2F0280EF76EF9
:1099C000C00EF66E81EC02F0EF6A65EC1DF012003D
:0699D00086EC45F01200D8
:020000040030CA
:03000100861A0F4D
:020005008181F7
:060008000FC00FE00F40E5
:00000001FF
